:020000040800F2
:10000000E80C002005A40008FDA4000801A50008D4
:1000100005A5000809A500080DA5000800000000BE
:1000200000000000000000000000000011A5000812
:1000300015A500080000000019A500081DA500086E
:1000400021A5000825A5000829A500082DA5000860
:1000500031A5000835A5000839A500083DA5000810
:100060004702000845A5000849A50008F50000085A
:1000700051A5000855A5000859A500085DA5000870
:1000800061A5000865A5000869A500086DA5000820
:1000900071A5000875A5000879A500087DA50008D0
:1000A00081A5000885A5000889A500088DA5000880
:1000B00091A5000895A50008B10100089DA50008BC
:1000C000A1A50008A5A50008A9A50008ADA50008E0
:1000D000B1A50008B5A50008B9A50008BDA5000890
:1000E0007D020008C5A50008C9A50008CDA5000827
:1000F000D1A5000880B5022001F0E9FF002202210D
:10010000774801F0D9FF7748008840280DDA764813
:100110000068764909880818734908607248406881
:10012000724949880818704948606E480088401C28
:100130006C49088001220221694801F0BDFF6C482A
:1001400002F00DF967480088402804DB00220221F4
:10015000634801F0B1FF01BD10B562480088402836
:1001600025DB00200400E4B2022C18DAE4B2614876
:1001700030F81400E4B25C4951F82410890911EBFD
:1001800040000321B0FBF1F0E4B25A4921F8140019
:10019000E4B25548002140F82410641CE3E75148BC
:1001A00000210180012202214D4801F085FF10BD90
:1001B00080B50121504802F09DF9002842D001216C
:1001C0004D4802F0B0F94D480078642815D14B48ED
:1001D000002101704A48012101700421494802F0C0
:1001E000FFF9002806D04848012101704748012145
:1001F000017002E044480021017045480088B0F5D4
:10020000FA7F05D142480021018042480121017056
:1002100041480088B0F5AF5F05D13F48002101801B
:100220003E480121017035480078401C3349087070
:1002300037480088401C3649088037480088401CF1
:100240003549088001BD80B5042002F04BFA002832
:1002500013D04FF4FA6002F06BFA4FF4FA6002F038
:1002600067FA042002F04BFA04212D4802F0B8F995
:10027000012802D12B480121017001BD80B54FF446
:10028000006002F02FFA002811D04FF4FA6002F05B
:100290004FFA4FF4006002F032FA4FF40061224846
:1002A00002F09EF9012802D11E48022101704FF48C
:1002B000004002F017FA002811D04FF4FA6002F063
:1002C00037FA4FF4004002F01AFA4FF400410D489B
:1002D00002F086F9012802D112480321017001BD04
:1002E00008600240C004002080040020B404002004
:1002F00000240140B004002000080040CC0400208D
:10030000CD04002000000240DB040020DC040020BB
:10031000C2040020CE040020C4040020CF0400202A
:10032000000C0240D0040020000802402DE9F043F8
:1003300093B0002400250CA8DFF8041D1C2202F055
:100340000FFA04A8DFF8FC1C0CC90CC008390838E7
:1003500002A8DFF8F41C0CC90CC00839083809A839
:10036000DFF8801E4CC94CC00C390C3806A8DFF8E9
:10037000781E4CC94CC00C390C38002602F01CFA0F
:1003800001F05CFB02F0D2FA032002F087FD0020AE
:1003900002F00FFD002001904FF6FF700090DFF893
:1003A0004C3EDFF84C2E5021322002F0B9FD0020E7
:1003B00001904FF6FF700090DFF8383EDFF8382EDE
:1003C00096210A2002F0ACFD002001904FF6FF704C
:1003D0000090DFF8203EDFF8282EB4210A2002F03A
:1003E0009FFD4FF47A7002F097F900200090C82327
:1003F00040F23F124E21082002F005FD002001903E
:100400004FF6FF700090DFF8EC3DDFF8402E1E2124
:100410001E2002F085FD04F00DF801F0AFFB01F0A5
:1004200059FC01F0C3FC01F005FD002001904FF6DE
:10043000FF700090DFF8BC3DDFF8142E64210A2025
:1004400002F06EFD4FF40071DFF8080E04F038FA88
:10045000DFF8041E0870DFF8043EDFF8042E4FF4C6
:100460000071DFF8F00D04F011FBDFF8EC1D0870EF
:10047000002001904FF6FF700090DFF8783DDFF824
:10048000E42D82210A2002F04BFD0222DFF8CC0D80
:10049000017889B20CA801F0A7FA0322DFF8BC0D9D
:1004A000417889B20DF1330001F09EFA0222DFF8A3
:1004B000AC0D817889B20DF1370001F095FA022276
:1004C000DFF8980DC17889B20DF13A0001F08CFA8D
:1004D0000222DFF8880D017989B20DF13D0001F0AB
:1004E00083FA0222DFF8740D417989B210A801F075
:1004F0007BFA0222DFF8640D817989B20DF14300A5
:1005000001F072FA0322DFF8540DC17989B20DF1BE
:10051000460001F069FA01220021012004F0CDF823
:10052000DFF8441D087002220021012004F0C5F804
:10053000DFF8381D087003220021012004F0BDF807
:10054000DFF82C1D087004220021012004F0B5F80A
:1005500005220021012004F0B0F8DFF8180D006832
:1005600004F024FB02000B00DFF80C1D04A804F0CB
:1005700045FBDFF8080D006804F018FB02000B00D3
:10058000DFF8F41C02A804F039FB002001904FF6BC
:10059000FF700090DFF85C3C0CAA9621192002F055
:1005A000BFFC4FF4C87001F0F3F9012002F0B4F879
:1005B0004FF4C87001F0ECF9012002F0ADF84FF4EF
:1005C000C87001F0E5F900200090C82340F23F1206
:1005D0001C21082002F017FC002002F0E1FF01209E
:1005E00002F0DEFFDFF8800C0178012003F078FCD8
:1005F000DFF8740E0078002800F06E85052001F009
:10060000C7F9DFF8640E0078012808D0C0F06185D2
:10061000032800F06382C0F0A78000F05ABDDFF825
:10062000500E0078042820D0DFF8480E007800280B
:100630000AD1DFF8400E012101704FF48051DFF83C
:10064000680E01F0DAFF8DE0DFF8280E007801284F
:1006500040F08880DFF81C0E002101704FF48051BB
:10066000DFF8440E01F0CBFF7CE0DFF8400E0078AD
:1006700000280DD1DFF83C0E0078012808D0DFF803
:10068000380E0078012803D0DFF8200E0121017018
:10069000DFF8200E007801282FD1DFF8200E007837
:1006A000401CDFF8181E0870DFF8100E00780528CF
:1006B00013D1DFF8080E0021017000200600002091
:1006C00000904E2340F209124E21C82002F0D6FCC1
:1006D000DFF8E00D002101700FE04FF4FC600090A6
:1006E0004E23F6B216F1E60292B24E21F6B216F1A0
:1006F000DC0080B202F0C2FC0A36DFF8BC0D0078E4
:1007000001282FD1DFF8B40D0078401CDFF8AC1DB4
:100710000870DFF8A80D0078052813D1DFF89C0DCC
:10072000002101700020060000200090622340F2AA
:1007300009126221C82002F0A1FCDFF87C0D002123
:1007400001700FE04FF4FC6000906223F6B216F1E6
:10075000E60292B26221F6B216F1DC0080B202F03B
:100760008DFC0A3600F0B5BCDFF8040D00780428D3
:100770002BD1DFF84C0D0078042826D1DFF8440D8A
:100780000078012821D1DFF83C0D00210170DFF84D
:10079000300D002101700122DFF8CC0A017889B206
:1007A000022003F08AFF0222DFF8C00A017889B232
:1007B000022003F082FF04220121022003F07DFFCA
:1007C00005220121022003F078FFDFF8A40C007855
:1007D000022807D10322DFF8980A017889B20220A3
:1007E00003F06BFFDFF8880C0078042811D1DFF8E4
:1007F000CC0C0021017000200600DFF8B80C0021AD
:100800000170DFF8B40C00210170DFF8BC0C00218E
:100810000170DFF85C0C0078401CDFF8541C087095
:10082000DFF84C0C0078052803DBDFF8440C0121CD
:100830000170DFF83C0C007802F0B2FEDFF8300CFB
:100840000078022840F0F580DFF8240A00780028BC
:1008500037D1002001904FF478400090DFF8503EEF
:10086000B2A2C52140F2111002F05AFB0020019003
:100870004FF6FF700090DFF8383EDFF8802ECF2172
:1008800040F2111002F04CFB002001904FF6FF7077
:100890000090DFF81C3EDFF8682ED92140F21110DD
:1008A00002F03EFB002001904FF6FF700090DFF851
:1008B000003EDFF8502EE32140F2111002F030FB31
:1008C0000BE1DFF8AC090078012837D10020019056
:1008D0004FF6FF700090DFF8D83D94A2C52140F29A
:1008E000111002F01DFB002001904FF478400090A1
:1008F000DFF8BC3DDFF8042ECF2140F2111002F0EA
:100900000FFB002001904FF6FF700090DFF8A03D34
:10091000DFF8EC2DD92140F2111002F001FB00208C
:1009200001904FF6FF700090DFF8843DDFF8D42D82
:10093000E32140F2111002F0F3FACEE0DFF83009C3
:100940000078022837D1002001904FF6FF70009008
:10095000DFF85C3D75A2C52140F2111002F0E0FA0B
:10096000002001904FF6FF700090DFF8443DDFF863
:100970008C2DCF2140F2111002F0D2FA002001900C
:100980004FF478400090DFF8283DDFF8742DD9212E
:1009900040F2111002F0C4FA002001904FF6FF70EF
:1009A0000090DFF80C3DDFF85C2DE32140F21110E0
:1009B00002F0B6FA91E0DFF8B8080078032840F0BA
:1009C0008C80002001904FF6FF700090DFF8E03C33
:1009D00056A2C52140F2111002F0A2FA00200190A7
:1009E0004FF6FF700090DFF8C83CDFF8102DCF21E4
:1009F00040F2111002F094FA002001904FF6FF70BF
:100A00000090DFF8AC3CDFF8F82CD92140F211104F
:100A100002F086FA002001904FF478400090DFF851
:100A2000903CDFF8E02CE32140F2111002F078FA5C
:100A300053E0DFF83C0A007803284ED1DFF8300895
:100A4000007800280ED1002001904FF478400090EB
:100A5000DFF85C3CDFF8182EC52140F2111002F0DF
:100A60005FFA3AE0DFF80808007801280ED100208C
:100A700001904FF478400090DFF8343CDFF8742E9A
:100A8000C52140F2111002F04BFA26E0DFF8E00732
:100A9000007802280ED1002001904FF47840009099
:100AA000DFF80C3CDFF8502EC52140F2111002F0A7
:100AB00037FA12E0DFF8B807007803280DD10020DC
:100AC00001904FF478400090DFF8E43BDFF8342CDD
:100AD000C52140F2111002F023FAFAE2DFF8900982
:100AE0000078042824D1DFF8CC09007801281FD031
:100AF000DFF8C409007801281AD0DFF8C4090078AB
:100B0000401CDFF8BC190870DFF8B409007805282C
:100B100003D1DFF8AC090021017000200090B4235C
:100B200011223721042002F06EF9D2E27831300030
:100B3000DFF880090078012840F0D480DFF87C09D4
:100B40000078002807D0022851D028D3042800F0CC
:100B5000A08075D3BDE2DFF81C07006804F026F81A
:100B60000022DFF80C3E04F063F804F0D5F8DFF85B
:100B700004170860DFF8FC06006804F017F800228C
:100B8000DFF8F43D04F010F90022DFF8E43D04F052
:100B90002FFA03D8DFF8DC060021016099E2DFF8C4
:100BA000D406006804F002F8DFF8D02DDFF8D03D5D
:100BB00004F03EF804F0B0F8DFF8B8160860DFF88B
:100BC000B4060068DFF8BC1D04F02AFA0ED8DFF87E
:100BD000A406006803F0EAFF0022DFF8E03D04F01D
:100BE00027F804F099F8DFF88C16086071E2DFF856
:100BF0008406006803F0DAFFDFF8C42DDFF8C43D97
:100C000004F016F804F088F8DFF868160860DFF8DA
:100C100064060068DFF8B01D04F002FA0FD8DFF8B0
:100C20005406006803F0C2FFDFF8502DDFF89C3D4A
:100C300003F0FEFF04F070F8DFF83816086048E2B1
:100C4000DFF83006006803F0B1FFDFF8842DDFF82D
:100C5000843D03F0EDFF04F05FF8DFF8181608603C
:100C6000DFF810060068DFF8701D04F0D9F90FD81E
:100C7000DFF80006006803F099FFDFF8442DDFF885
:100C80005C3D03F0D5FF04F047F8DFF8E815086095
:100C90001FE2DFF8E005006803F088FFDFF8402D71
:100CA000DFF8403D03F0C4FF04F036F8DFF8C41568
:100CB0000860DFF8C0050068DFF8CC1C04F0B0F96C
:100CC0000FD8DFF8B005006803F070FFDFF8002DE3
:100CD000DFF8B83C03F0ACFF04F01EF8DFF8941521
:100CE0000860F6E1DFF8D0070078012840F0D480F2
:100CF000DFF8C8070078002807D0022851D028D391
:100D0000042800F0A08075D3E3E1DFF870050068E7
:100D100003F04CFF0022DFF8583C03F089FF03F09A
:100D2000FBFFDFF858150860DFF85005006803F096
:100D30003DFF0022DFF8403C04F036F80022DFF8E7
:100D4000303C04F055F903D8DFF83005002101608C
:100D5000BFE1DFF82805006803F028FFDFF81C2C4E
:100D6000DFF81C3C03F064FF03F0D6FFDFF80C153E
:100D70000860DFF808050068DFF8081C04F050F987
:100D80000ED8DFF8F804006803F010FF0022DFF847
:100D90002C3C03F04DFF03F0BFFFDFF8E0140860C8
:100DA00097E1DFF8D804006803F000FFDFF8102CAB
:100DB000DFF8103C03F03CFF03F0AEFFDFF8BC149B
:100DC0000860DFF8B8040068DFF8FC1B04F028F9BD
:100DD0000FD8DFF8A804006803F0E8FEDFF89C2BCA
:100DE000DFF8E83B03F024FF03F096FFDFF88C14F4
:100DF00008606EE1DFF88404006803F0D7FEDFF8D6
:100E0000D02BDFF8D03B03F013FF03F085FFDFF8B2
:100E10006C140860DFF864040068DFF8BC1B04F0A1
:100E2000FFF80FD8DFF85404006803F0BFFEDFF8C6
:100E3000902BDFF8A83B03F0FBFE03F06DFFDFF81B
:100E40003C14086045E1DFF83404006803F0AEFEAE
:100E5000DFF88C2BDFF88C3B03F0EAFE03F05CFF3D
:100E6000DFF818140860DFF814040068DFF8181BB6
:100E700004F0D6F80FD8DFF80404006803F096FEFB
:100E8000DFF84C2BDFF8043B03F0D2FE03F044FF05
:100E9000DFF8E81308601CE1DFF8D40500780228C9
:100EA00040F01781DFF8C8030078002840D1DFF850
:100EB000C00301210170DFF8B805007802F070FB73
:100EC000002001904FF6FF700090DFF8E437CBA2CE
:100ED000C52140F2111002F023F8002001904FF4D8
:100EE00078400090DFF8C837DFF81028CF2140F2B3
:100EF000111002F015F8002001904FF6FF700090DD
:100F0000DFF8AC37DFF8F827D92140F2111002F0F2
:100F100007F8002001904FF6FF700090DFF890373F
:100F2000DFF8E027E32140F2111001F0F9FFD0E0F3
:100F3000CF48007801283FD1CD4802210170DFF869
:100F40003005007802F02CFB002001904FF6FF7076
:100F50000090DFF85C37A9A2C52140F2111001F022
:100F6000DFFF002001904FF6FF700090DFF8403760
:100F7000DFF88827CF2140F2111001F0D1FF0020C7
:100F800001904FF478400090DFF82437DFF87027A5
:100F9000D92140F2111001F0C3FF002001904FF65B
:100FA000FF700090DFF80837DFF85827E32140F2A0
:100FB000111001F0B5FF8CE0AD480078022845D152
:100FC000AB4803210170DFF8A804007802F0E8FACA
:100FD000002001904FF6FF700090DFF8D43687A212
:100FE000C52140F2111001F09BFF002001904FF647
:100FF000FF700090DFF8B836DFF80027CF2140F20D
:10100000111001F08DFF002001904FF6FF7000904D
:10101000DFF89C36DFF8E826D92140F2111001F004
:101020007FFF002001904FF478400090DFF8803679
:10103000DFF8D026E32140F2111001F071FF48E003
:10104000887400085CA4000864A40008884800783C
:1010500003283ED1864800210170DFF8140400788F
:1010600002F09EFA002001904FF478400090DFF8E3
:10107000403662A2C52140F2111001F051FF00205C
:1010800001904FF6FF700090DFF82436DFF86C26F1
:10109000CF2140F2111001F043FF002001904FF6E4
:1010A000FF700090DFF80836DFF85426D92140F2AF
:1010B000111001F035FF002001904FF6FF700090F5
:1010C000DFF8EC35DFF83C26E32140F2111001F0A7
:1010D00027FFE54800210170DFF8F40B00780128B4
:1010E00040F03A84DFF8E80B00210170DFF8B00C23
:1010F0000078012820D1002001904FF47840009022
:101100003C4BDAA2462140F21D1001F009FF57487E
:10111000007801282AD1D7480078012807D1D5487E
:10112000002101704FF48051DF4801F068FA4FF45C
:101130007A7000F02DFC19E0DFF8640C00780028CC
:1011400014D1DFF8600C007801280FD10020019045
:101150004FF4FC600090274BD5A2462140F21D10B1
:1011600001F0DEFEDFF83C0C00210170C148007880
:10117000012825D1DFF8300C007800280CD1DFF8E9
:10118000280C012101704FF4FC6308222F214FF439
:10119000937002F06CF848E0DFF80C0C007801283E
:1011A00043D1DFF8040C00210170002000903823A7
:1011B00040F22F12262140F21D1001F024FE34E0EF
:1011C000DFF8E40B007800281CD1DFF8DC0B0121EC
:1011D00001704FF4784308222F214FF4937002F0EE
:1011E00046F822E014A4000820A400080C01002006
:1011F000A4A300080401002010A3000878313000E7
:1012000030A30008DFF8A00B007801280DD1DFF82B
:10121000980B0021017000200090382340F22F121B
:10122000262140F21D1001F0EEFDFEF795FF9048DB
:101230000078012824D0C0F08F83032800F0868135
:10124000C0F04481042800F0038285E3B4A30008C1
:101250007CA3000800040240D5040020880400207C
:10126000D604002090A30008D7040020DD0400204D
:10127000DF040020140100206CA4000818010020E5
:10128000DFF82C0C408803F0DDFEDFF8281C03F0AB
:10129000E9FE03F08BFCDFF8202CDFF8203C03F0A4
:1012A0004DFF0022DFF8183C03F07EFD80468946A2
:1012B000DFF8100C006803F079FC02000B004046D8
:1012C000494603F071FD03F027FD040002221700D8
:1012D000200004F005F880B24FF47A7190FBF1F130
:1012E0003A0089B209A800F07FFB200003F0F8FF64
:1012F00080B24FF47A71032290FBF1F301FB1301EA
:1013000089B20DF1270000F06FFB002001904FF42F
:10131000FC600090DFF8B03B09AA5021462001F0A4
:10132000FFFD54480078012840F0A680664800215F
:101330000170DFF87C0B008803F0FEFF0022DFF86D
:101340008C3B03F075FCDFF8882BDFF8883B03F05B
:101350002BFD80468946DFF8800B006803F026FCF1
:1013600002000B004046494603F01EFD03F0D4FC8A
:101370000500280003F0B4FF80B247F230518842E4
:1013800064DA02221700280003F0AAFF80B242F2BA
:10139000107190FBF1F13A0089B206A800F024FB2D
:1013A000280003F09DFF80B242F21071042290FBEE
:1013B000F1F301FB130189B20DF11B0000F014FBE6
:1013C000002001904FF4FC600090DFF8FC3A06AA80
:1013D0008C21462001F0A4FD280003F081FF80B29B
:1013E00003F0AAFF0022DFF8F43A03F0A7FE002280
:1013F000DFF8EC3A03F0D8FC03F0ACFF00B201F0E8
:10140000DCFFDFF8E00A00780090002300221700DC
:101410009846280003F064FF010043463A0089B271
:10142000022002F0CAFDDFF8BC0A00780090002319
:10143000002217009846200003F052FF01004346A7
:101440003A0089B2012002F0B8FD2CE000200190A2
:101450004FF478400090DFF8703ADFF88C2A8C2146
:10146000462001F05DFD1EE0D00400204343000053
:1014700020010020D804002013480078002812D151
:10148000002001904FF4FC600090DFF83C3ADFF858
:10149000582A8C21462001F043FD002001F08DFFE9
:1014A00009480121017057E200000240D2040020E7
:1014B00043560000D3040020D4040020E0040020A0
:1014C000D1040020DE040020DA040020DFF81C0A2A
:1014D0000078012839D1DFF8D809008803F02CFF03
:1014E0000022DFF8E83903F0A3FBDFF8E429DFF896
:1014F000E43903F059FC80468946DFF8DC090068CE
:1015000003F054FB02000B004046494603F04CFC3C
:1015100003F002FC0500280003F0E2FE80B247F26F
:101520003051884211DADFF8BC09007800900023BE
:10153000012217009846280003F0D2FE010043461E
:101540003A0089B2022002F038FD05E2DFF89C097A
:10155000007801287BD1DFF85809408803F072FD3C
:10156000DFF8501903F07EFD03F020FBDFF8482977
:10157000DFF8483903F0E2FD0022DFF8443903F0D8
:1015800013FC80468946DFF83C09006803F00EFB37
:1015900002000B004046494603F006FC03F0BCFB8A
:1015A0000400DFF8400900780090002300221700B3
:1015B0009846200003F094FE010043463A0089B2A9
:1015C000012002F0FAFCDFF8E808008803F0B4FE1E
:1015D0000022DFF8F83803F02BFBDFF8F428DFF8FF
:1015E000F43803F0E1FB80468946DFF8EC08006838
:1015F00003F0DCFA02000B004046494603F0D4FB3E
:1016000003F08AFB0500DFF8DC0800780090002377
:10161000002217009846280003F062FE01004346AE
:101620003A0089B2022002F0C8FCDFF8B80800785E
:1016300000900123012217009846280003F050FE75
:10164000010043463A0089B2032002F0B6FC83E170
:10165000DFF89C080078002807D0022854D029D34E
:10166000042800F0998073D3B9E0002001904FF670
:10167000FF700090DFF8B837BEA23C21052001F0D2
:101680004FFCDFF870080078012810D1DFF86408FB
:1016900000210170DFF86008012101704FF4FC6047
:1016A00000904E23D2224E21C82001F0E7FC96E0A4
:1016B000FC000020002001904FF6FF700090DFF842
:1016C0007037ACA25021052001F02AFCDFF8240875
:1016D0000078012810D1DFF81C0800210170DFF824
:1016E0001C08012101704FF4FC6000906223D2229B
:1016F0006221C82001F0C2FC71E000BF74A40008A0
:101700007CA4000884A40008002001904FF6FF701C
:101710000090DFF81C3797A26421052001F000FC3F
:10172000DFF8D0070078012811D1DFF8C8070021C1
:101730000170DFF8CC070078002804D1DFF8C0077B
:101740000121017003E0DFF8B8070021017046E0D5
:10175000002001904FF6FF700090DFF8D43685A28C
:101760007821052001F0DCFBDFF8880700780128EC
:1017700011D1DFF8800700210170DFF888070078B9
:10178000002804D1DFF87C070121017003E0DFF8B5
:1017900074070021017022E0002001904FF6FF70D5
:1017A0000090DFF88C3673A28C21052001F0B8FB85
:1017B000DFF840070078012811D1DFF83807002151
:1017C0000170DFF844070078002804D1DFF83807FB
:1017D0000121017003E0DFF8300700210170DFF81C
:1017E00018070078012818D1DFF8D806006803F040
:1017F000DDF902000B00DFF8141704A803F0FEF96E
:10180000002001904FF478400090DFF8243604AABD
:101810003C21C82001F084FB0BE0002001904FF632
:10182000FF700090DFF8083604AA3C21C82001F0C0
:1018300077FBDFF8C806007801281BD1DFF898068F
:10184000006803F0B3F902000B00DFF8C01602A82D
:1018500003F0D4F9002001904FF478400090DFF8B5
:10186000D03502AA5021C82001F05AFB0EE000BF7B
:101870008CA40008002001904FF6FF700090DFF864
:10188000B03502AA5021C82001F04AFBDFF87006EB
:10189000007800280CD1002001904FF6FF700090D6
:1018A000DFF88C35B1A26421DC2001F039FB0BE0BC
:1018B000002001904FF6FF700090DFF87435ACA265
:1018C0006421DC2001F02CFBDFF8380600780028CA
:1018D00014D1002001904FF6FF700090DFF85035D2
:1018E000A2A27821DC2001F01BFB0021012002F0E4
:1018F000F7FA13E094A400089CA4000800200190CB
:101900004FF6FF700090DFF8283599A27821DC208F
:1019100001F006FB0121012002F0E2FADFF8E80500
:10192000007800280CD1002001904FF6FF70009045
:10193000DFF8FC348FA28C21DC2001F0F1FA0BE0FF
:10194000002001904FF6FF700090DFF8E4348AA287
:101950008C21DC2001F0E4FADFF8B40500780128DE
:101960007EF446AEDFF8A80500210170FEF740BE08
:101970000000F03F3E000000000024409A99999931
:101980009999B93F67661E4198FF1F414D6250BF4C
:1019900010B50400DFF86C05007801280DD108218E
:1019A000DFF8700500F02BFEA4B2200000F0B4FEBA
:1019B0000821DFF8600500F020FE10BD000024C003
:1019C0007B14AE47E17A843F0BD71F419999B9BF89
:1019D000FCA9F1D24D62503FE8FB1F41E17A84BF80
:1019E0002D431CEBE2361A3F7EB400242300DBB209
:1019F000D2B2934213D289B20A24D2B2DBB2D51A40
:101A000000AEAD1991FBF4F604FB1614303405F862
:101A1000014C89B20A2491FBF4F15B1CE7E7002436
:101A20002300DBB2D2B2934206D2DBB2DBB200AC0F
:101A30001C5D1C545B1CF4E777BC704780B501212A
:101A40000D2003F0B8FCDFF8D00408210160DFF8B6
:101A5000C80401210171DFF8C00400218171DFF8A1
:101A6000B8040121C171DFF8B014DFF8A80400F058
:101A700063FD0821DFF89C0400F0BFFDDFF8980447
:101A80004FF480510160DFF8900401210171DFF80B
:101A9000880400218171DFF880040021C171DFF822
:101AA0007814DFF8700400F047FD4FF48051DFF840
:101AB000640400F0A4FDDFF8600404210160DFF895
:101AC000580400210171DFF8500400218171DFF812
:101AD00048040021C171DFF84014DFF8380400F039
:101AE0002BFDDFF8340404210160DFF82C04002111
:101AF0000171DFF8240400218171DFF81C04022148
:101B0000C171DFF81414DFF8140400F015FDDFF8DC
:101B100008044FF400610160DFF8FC03002101714B
:101B2000DFF8F40300218171DFF8EC030221C171B9
:101B3000DFF8E413DFF8E80300F0FEFCDFF8D80379
:101B40004FF400410160DFF8D00300210171DFF89C
:101B5000C80300218171DFF8C0030221C171DFF8E1
:101B6000B813DFF8B00300F0E7FC01BD4F464600B4
:101B70004F4E20004E4F20005945530080B50121A3
:101B8000022003F018FC01215FF0807003F013FCC9
:101B9000DFF8840303210160DFF87C030321017176
:101BA000DFF874030021C171DFF86C13DFF87403F0
:101BB00000F0C2FCDFF8700300F0CCF9DFF86C0332
:101BC000DFF86C130160DFF86403DFF8681341602D
:101BD000DFF8580300218160DFF850030221C16063
:101BE000DFF8480300210161DFF8400380214161F3
:101BF000DFF838034FF480718161DFF830034FF470
:101C00008061C161DFF8240320210162C7484FF4DD
:101C100000514162C54800218162C449C24800F0B8
:101C20001EFA0121C04800F039FA01220221BE4803
:101C300000F042FA012003F0B9FB212003F0E8FB99
:101C40000028FAD001214FF4007003F0C3FBBA481A
:101C500000210160B84801210171B748002141719C
:101C6000B54800218160B4480021C160B24800211C
:101C70000161B14802210175AF49B04800F04CFA4A
:101C8000072301220821AD4800F08AFA0723022227
:101C90000921AA4800F084FA0121A84800F071FB4C
:101CA00001225FF44031A54800F06BFA0121A348FE
:101CB00000F05AFB0121A14800F056FA40219F484C
:101CC00000F06CFB0028F9D09C4800F048FB01BDF7
:101CD000CE04002080B50121012003F08AFB012100
:101CE000012003F068FB8C48022101608A48022130
:101CF00001718948012141718749864800F01CFC27
:101D000001220121834800F07CFC8D4800F096FB05
:101D10008B4840F23F114160894800210180884989
:101D20005FF0804000F058FB8648602101808548C4
:101D300001214180834800210181824801214180A5
:101D40008048642141607F495FF0804000F09CFB47
:101D500008215FF0804000F0B8FB01215FF0804077
:101D600000F076FB01215FF0804000F07FFB012155
:101D7000042003F03EFB724847F6FF414160704883
:101D8000002101806E49704800F026FB01216E4859
:101D900000F06CFB012201216B4800F0A0FB01BDAB
:101DA000DB040020DC040020D904002080B50121E0
:101DB000012003F00FFB0221032003F057FB6348CF
:101DC00004210160614800210171604808214171CE
:101DD0005E48012181715D4800F040FC0B2102202A
:101DE00003F044FB59484FF400610160574800215B
:101DF00001715648082141715448012181715348AD
:101E000000F02CFC0F21002003F030FB4F484FF472
:101E1000004101604D48002101714C480821417189
:101E20004A4801218171494800F018FC01BD0000B9
:101E30000401002080B546480B210170444801216F
:101E4000417043480021817041480121C1704048E0
:101E500003F036FB3E481E2101703D4800214170D1
:101E60003B48002181703A480121C170384803F095
:101E700027FB37480821017035480021417034485C
:101E80000221817032480121C170314803F018FBF2
:101E90002F48282101702E48002141702C48012133
:101EA00081702B480121C170294803F009FB01BD55
:101EB000B004002000304D45CDCCCCCCCCCC25405E
:101EC0000000B040140100200C010020000018C0E8
:101ED000B81E85EB51B8BE3F1801002000005940E4
:101EE000004CDD40DF0400202CA40008D8040020B2
:101EF000D1040020D2040020D3040020D404002008
:101F0000DD040020D7040020DE0400206CA40008BB
:101F1000CF0400200000024090040020000C02408A
:101F20000008024000040240086002401C04002037
:101F300058240140B404002048040020002401403B
:101F4000600400206C040020000800409804002079
:101F5000B804002001684FF6FE72114001600021B4
:101F6000016000214160002181600021C1605C4965
:101F7000884206D15B49096851F00F01594A116046
:101F80006CE05949884206D15649096851F0F00180
:101F9000544A116062E05549884206D151490968A6
:101FA00051F470614F4A116058E05149884206D19E
:101FB0004C49096851F470414A4A11604EE04D495C
:101FC000884206D14749096851F47021454A116099
:101FD00044E04949884206D14249096851F47001F8
:101FE000404A11603AE04549884206D13D490968B6
:101FF00051F070613B4A116030E04149884206D19E
:102000004049096851F00F013E4A116026E03E49FF
:10201000884206D13B49096851F0F001394A116004
:102020001CE03A49884206D13649096851F470618A
:10203000344A116012E03649884206D131490968B4
:1020400051F470412F4A116008E03249884205D1AD
:102050002C49096851F470212A4A1160704710B464
:10206000002203681A006FF30E128B680C6A234378
:102070000C6923434C6923438C692343CC69234374
:102080004C6A23438C6A23431A430260CB68436043
:102090000B6883604B68C36010BC7047C9B20029ED
:1020A00004D0026852F00102026004E002684FF6B8
:1020B000FE731A4002607047D2B2002A03D0036850
:1020C0000B43036002E003688B4303607047C10069
:1020D00002D40449086001E00A4908607047000022
:1020E00008600240046002401C6002403060024010
:1020F00044600240586002406C60024080600240D0
:1021000008640240046402401C64024030640240DF
:10211000446402405864024030B400230022446802
:1021200023001D4C23400C790D6855EA04242343F9
:10213000436084682300194C23400C69CD682C430C
:102140008D682C434D7954EA450423438360046B26
:10215000230033F0F8730C7D641E2243D2B253EA9D
:102160000253036330BC7047C9B2002904D08268AF
:1021700052F00102826003E08268520852008260DD
:102180007047D2B2002A03D043680B43436002E099
:1021900043688B4343607047FFFEFFFCFDF7FFC0C1
:1021A000F0B400250024C9B21E2916DBC66D350027
:1021B0000726B1F11E075FF0030C0CFB07F7BE40CA
:1021C0003400A543DBB2B1F11E0603277E4313FAA8
:1021D00006F634002543C56545E0C9B2142916DB6F
:1021E000C66835000726B1F114075FF0030C0CFB3D
:1021F00007F7BE403400A543DBB2B1F11406032754
:102200007E4313FA06F634002543C5602BE0C9B2BD
:102210000A2916DB066935000726B1F10A075FF0C7
:10222000030C0CFB07F7BE403400A543DBB2B1F151
:102230000A0603277E4313FA06F634002543056198
:1022400011E0466935000726032707FB01F7BE406A
:102250003400A543DBB2032606FB01F613FA06F6AB
:10226000340025434561D2B2072A14DA066C3500E2
:102270001F26571E5FF0050C0CFB07F7BE4034000D
:10228000A543C9B2561E05277E4311FA06F634004F
:102290002543056461E0D2B20D2A14DAC66B35001D
:1022A0001F26D71F5FF0050C0CFB07F7BE4034005C
:1022B000A543C9B2D61F05277E4311FA06F634009E
:1022C0002543C56349E0D2B2132A16DA866B35007E
:1022D0001F26B2F10D075FF0050C0CFB07F7BE409F
:1022E0003400A543C9B2B2F10D0605277E4311FAA9
:1022F00006F63400254385632FE0D2B2192A16DA98
:10230000466B35001F26B2F113075FF0050C0CFB7E
:1023100007F7BE403400A543C9B2B2F11306052742
:102320007E4311FA06F634002543456315E0066B3B
:1023300035001F26B2F119075FF0050C0CFB07F7FB
:10234000BE403400A543C9B2B2F1190605277E4349
:1023500011FA06F6340025430563F0BC7047816826
:1023600051F0804181607047C9B2002904D0826871
:1023700052F48072826003E0826832F4807282607C
:102380007047C9B2002904D0826852F4007282609A
:1023900003E0826832F4007282607047020000201D
:1023A000136889B20B4202D00123180001E0002318
:1023B0001800C0B2704750F8041B61B150F8042BEC
:1023C000D30744BFA9F101039A18002342F8043B44
:1023D000091FFAD1EFE77047002203881A00B0F115
:1023E000804F08D0104B984205D0104B984202D035
:1023F0000F4B984204D14FF68F731A404B881A4303
:102400000C4B984207D00C4B984204D04FF6FF4338
:102410001A400B891A4302804B68C3620B880385FC
:102420000123838270470000000400400008004040
:10243000000C004000100040001400405FF0FF312D
:10244000416000210180002101810021418070470D
:10245000C9B2002904D0028852F08002028004E050
:1024600002884FF67F731A4002807047C9B2002974
:1024700004D0028852F00102028004E002884FF684
:10248000FE731A400280704730B400220023048C8F
:102490004FF6EF752C400484048C2300048B22003B
:1024A00048F6FF7422400C8852EA04224FF6DF748B
:1024B00023400C8953EA04134C8853EA04134C68F4
:1024C00084630283038430BC70470022038B1A00AC
:1024D0004FF2FF731A4052EA012202837047D2B2D0
:1024E000002A03D083890B43838102E083898B43D5
:1024F0008381704730B40200002000230024158A35
:102500000D402B0095890D402C009BB2002B05D06F
:10251000A4B2002C02D00125280001E000252800EB
:10252000C0B230BC704789B2CA43028270470268A9
:10253000531C036011707047F0B400220023002484
:1025400000252A00102A49D2012595402B000D684C
:102550001D402C009C423FD1056803261700FFB2A6
:102560007F00BE40B543056005680E791700FFB2D5
:102570007F00BE40354305600D79012D02D00D79F5
:10258000022D19D1856803261700FFB27F00BE40D7
:10259000B543856085684E791700FFB27F00BE4065
:1025A00035438560858801269640B54385808588BA
:1025B0008E79964035438580C56803261700FFB2A3
:1025C0007F00BE40B543C560C568CE791700FFB235
:1025D0007F00BE403543C560521CB3E7F0BC704776
:1025E00002000020138A89B20B4202D00123180096
:1025F00001E000231800C0B2704701837047418397
:102600007047F0B400230024D2B211F00705EDB2F8
:10261000AD0012FA05F52B0089B2CD1010EB85053F
:1026200089B2CE1010EB8606366A0F2711F0070C20
:102630005FFA8CFC5FEA8C0C17FA0CF7BE432E6233
:1026400089B2CD1010EB85052D6A1D432C0089B28F
:10265000CD1010EB85052C62F0BC70470021294A93
:1026600011008279002A36D0264A126803689A43FC
:10267000244B1A60244A126803689A43224B1A605A
:10268000027951180A6803681A430A601F4A1268DF
:1026900003689A431D4B1A601D4A126803689A43E7
:1026A0001B4B1A604279102A0CD1184A1268036831
:1026B0001A43164B1A60164A126803681A43144BE1
:1026C0001A600EE00F4A1100427951180A68036837
:1026D0001A430A6005E0027951180A6803689A43B0
:1026E0000A607047010000200A4A12680A4202D0BC
:1026F0000122100001E000221000C0B2704705491D
:1027000008607047000401400404014008040140CF
:102710000C040140140401404FF47A61034A01FBA8
:102720000020002801D0401EFBE7704740420F0008
:1027300005214843002801D0401EFBE770470000F8
:1027400062B38B0708D0521E11F8013B00F8013B21
:1027500000F024808B07F6D1830740F0208000BF73
:10276000103A07D330B4B1E83810103AA0E8381066
:10277000F9D230BC530724BFB1E80810A0E8081014
:1027800044BF51F8043B40F8043BD20724BF31F862
:10279000022B20F8022B44BF0B7803707047083AD5
:1027A00007D3B1E80810083A40F8043B40F804CBDE
:1027B000F7D25307E4E7000080B55248006850F4B0
:1027C00080705049086050480068504908404E49A0
:1027D00008604C4800684E4908404A49086049482A
:1027E000006830F48020474908604748006830F4AA
:1027F0007D004549086047480021016000F005F868
:1028000045485FF00061016001BD82B00020019089
:10281000002000903B48006850F48030394908603F
:102820003848006810F4003000900198401C019076
:102830000098002803D10198B0F5A06FF0D131487D
:102840000068800302D50120009001E00020009084
:102850000098012853D13148006850F004002F49F6
:1028600008602E48006850F002002C4908602B4890
:10287000006850F00100294908602948006850F0BC
:1028800080502749086027484FF4006101602648BE
:102890000068C006FBD41C481B49096801601A483F
:1028A0001949096801601848174909680160164804
:1028B000006830F47D00144908601348006850F443
:1028C0001100114908600F48006850F080700D49F0
:1028D00008600C4800688001FBD50B480068800840
:1028E0008000094908600848006850F00300064964
:1028F00008600548006810F00C000C28F9D102B0FF
:102900007047000000380240083802400CC0FF88C1
:10291000FEFFFEEE0C38024008ED00E0003C0240F5
:1029200024380240007000400470004000B587B0B9
:102930000121022002F03FFD4FF4E0500090012001
:102940008DF8040003208DF8050000208DF80600A6
:1029500000208DF8070000A9DFF84C08FFF7ECFD18
:102960004FF46040009002208DF8040003208DF8A1
:10297000050000208DF8060000208DF8070000A952
:10298000DFF82408FFF7D8FD05220D21DFF818082D
:10299000FFF737FE05220E21DFF80C08FFF731FEA6
:1029A00005220F21DFF80008FFF72BFE01214FF46D
:1029B000804002F01EFD4FF48270ADF80A00002046
:1029C000ADF808000820ADF814000020ADF80E00A6
:1029D0000020ADF810000020ADF816000020ADF882
:1029E0000C004FF40070ADF812000020ADF8180094
:1029F00002A9DFF8B80702F0A1FD0121DFF8AC075A
:102A000002F0BCFD4FF48051DFF89C07FFF7F5FDA5
:102A100000F01AF80020DFF898170880DFF8941704
:102A20000880DFF89407F0210180DFF88C074FF46D
:102A3000A0714180DFF88007012101714FF6FF701E
:102A400000F0B7F907B000BD80B54FF48061DFF842
:102A50005807FFF7D4FDDFF8640700F015FA4FF4CC
:102A60008061DFF84407FFF7C8FD012000F020F97E
:102A7000DFF8480700F008FACB2000F019F93920F8
:102A800000F031F92C2000F02EF9002000F02BF995
:102A9000342000F028F9022000F025F9CF2000F0C2
:102AA00007F9002000F01FF9C12000F01CF93020C8
:102AB00000F019F9E82000F0FBF8852000F013F988
:102AC000002000F010F9782000F00DF9EA2000F065
:102AD000EFF8002000F007F9002000F004F9ED20E5
:102AE00000F0E6F8642000F0FEF8032000F0FBF8A8
:102AF000122000F0F8F8812000F0F5F8F72000F03F
:102B0000D7F8202000F0EFF8C02000F0D1F8232003
:102B100000F0E9F8C12000F0CBF8102000F0E3F855
:102B2000C52000F0C5F83E2000F0DDF8282000F0B8
:102B3000DAF8C72000F0BCF8862000F0D4F8362080
:102B400000F0B6F8482000F0CEF83A2000F0B0F8D7
:102B5000552000F0C8F8B12000F0AAF8002000F0DD
:102B6000C2F8182000F0BFF8B62000F0A1F8082045
:102B700000F0B9F8822000F0B6F8272000F0B3F892
:102B8000F22000F095F8002000F0ADF82A2000F0C7
:102B90008FF8002000F0A7F8002000F0A4F8002033
:102BA00000F0A1F8EF2000F09EF82B2000F080F854
:102BB000002000F098F8002000F095F8012000F0C7
:102BC00092F83F2000F08FF8262000F071F80120E5
:102BD00000F089F8E02000F06BF80F2000F083F897
:102BE000312000F080F82B2000F07DF80C2000F060
:102BF0007AF80E2000F077F8082000F074F84E20E4
:102C000000F071F8F12000F06EF8372000F06BF85A
:102C1000072000F068F8102000F065F8032000F0AD
:102C200062F80E2000F05FF8092000F05CF8002048
:102C300000F059F8E12000F03BF8002000F053F8D4
:102C40000E2000F050F8142000F04DF8032000F0A2
:102C50004AF8112000F047F8072000F044F831202E
:102C600000F041F8C12000F03EF8482000F03BF8A9
:102C7000082000F038F80F2000F035F80C2000F0A4
:102C800032F8312000F02FF8362000F02CF80F2019
:102C900000F029F8112000F00BF8DFF8FC0800F034
:102CA000F3F8292000F004F82C2000F001F801BD11
:102CB00010B504004FF40061DFF8EC04FFF79FFC4F
:102CC0004FF48051DFF8E004FFF799FC2100C9B20E
:102CD000DFF8D80402F070FC4FF48051DFF8C8042C
:102CE000FFF78BFC10BD10B504004FF40061DFF856
:102CF000B804FFF782FC4FF48051DFF8AC04FFF713
:102D00007EFC2100C9B2DFF8A40402F055FC4FF4A8
:102D10008051DFF89404FFF770FC10BD70B504001B
:102D20000D0016002B009BB2220092B2290089B23E
:102D3000200080B200F00DF82C20FFF7B9FFB6B2EA
:102D4000300AC0B2FFF7CFFF3000C0B2FFF7CBFFB1
:102D500070BDF8B504000D0016001F002A20FFF713
:102D6000A7FFA4B2200AC0B2FFF7BDFF2000C0B287
:102D7000FFF7B9FFB6B2300AC0B2FFF7B4FF3000B8
:102D8000C0B2FFF7B0FF2B20FFF792FFADB2280AC9
:102D9000C0B2FFF7A8FF2800C0B2FFF7A4FFBFB280
:102DA000380AC0B2FFF79FFF3800C0B2FFF79BFFA1
:102DB000F1BDF8B50400A4B2200A80B20600A4B2A6
:102DC000E0B20700DFF8F0034088431E9BB2DFF853
:102DD000E8030088421E92B200210020FFF7B9FFED
:102DE0002C20FFF765FF00200500B5F5963F09D2BE
:102DF0003000C0B2FFF777FF3800C0B2FFF773FFB3
:102E00006D1CF2E7F1BD2DE9F84F05000E0017002B
:102E100098460A9CBFB2ADB2AF4204D31FFA88F8FD
:102E2000B6B2B04500D2FEE7BFB2ADB2781B1FFA12
:102E300088F8B6B2B8EB060148438346A4B2200A2C
:102E400080B20090A4B2E0B28246B8F101039BB216
:102E50007A1E92B2310089B2280080B2FFF779FF62
:102E60002C20FFF725FF00208146D9450AD2009883
:102E7000C0B2FFF738FF5046C0B2FFF734FF19F178
:102E80000109F2E7BDE8F18F01B40098002803D0F2
:102E90000098401E0090F8E701B0704710B504009C
:102EA0003620FFF705FFE4B2002C03D15820FFF7CE
:102EB0001AFF13E0E4B2012C03D18820FFF713FFBF
:102EC0000CE0E4B2022C03D12820FFF70CFF05E050
:102ED000E4B2032C02D1E820FFF705FFE4B2002C96
:102EE00002D0E4B2012C0DD1DFF8B006F021018050
:102EF000DFF8A8064FF4A0714180DFF8A006012199
:102F000001710CE0DFF894064FF4A0710180DFF846
:102F10008C06F0214180DFF884060021017110BD8C
:102F20002DE9FC4706000F00904699460A9C0B9D30
:102F3000B246A04806809E48078098F80000002806
:102F400032D098F800000A2817D19948008899F8DB
:102F50000110491C08189649088098F801000D28AE
:102F600005D194480021018018F1010802E0914840
:102F7000A0F800A018F10108DFE798F800000D287C
:102F800002D118F10108D8E7ADB20195A4B20094BE
:102F90004B4698F80020864801888648008800F053
:102FA00005F818F10108C8E7BDE8F3872DE9F14FEE
:102FB0000E00170098460A9C0B9D7E48BDF8001035
:102FC00001807B4806807C4800887A49098898F807
:102FD00000205118884209DA7548008898F80110D5
:102FE0000818734908807348002101800020814639
:102FF00098F80100814538D2FFB2B7F1200098F867
:10300000011001FB0090D8F8041031F8100082463E
:103010000020834698F80000834523D21AFA0BF06B
:1030200000040ED5220092B26148008819EB00011D
:1030300089B2604800881BEB000080B2FFF76EFE8B
:103040000DE02A0092B25A48008819EB000189B2BB
:10305000584800881BEB000080B2FFF75FFE1BF1B1
:10306000010BD7E719F10109C2E75248008898F827
:10307000001008184F490880BDE8F18F2DE9F84F7E
:1030800004000D0016001F00DFF810050088A4B230
:10309000844204D3DFF804050088401E0400DFF8F2
:1030A000FC040088B6B2864204D3DFF8F00400883E
:1030B000401E0600DFF8E4044088ADB2854204D328
:1030C000DFF8D8044088401E0500DFF8D0044088AF
:1030D000BFB2874204D3DFF8C4044088401E070013
:1030E000A4B2B6B2B44202D2B6EB040A01E0B4EB29
:1030F000060AADB2BFB2BD4202D2B7EB050B01E08A
:10310000B5EB070BA4B2B6B2B44201D2012001E084
:103110005FF0FF30ADF80200ADB2BFB2BD4201D2E8
:10312000012001E05FF0FF30ADF800000FFA8BFBEB
:103130000FFA8AFAD34503DA0FFA8AFA504603E007
:103140000FFA8BFBDBF10000022190FBF1F8BDF8D8
:103150002820290089B2200080B2FFF7DFFDA4B249
:10316000B6B2B44203D1ADB2BFB2BD4219D0C1466E
:103170000FFA8AFADAF100000FFA89F9484504DA01
:10318000B8EB0B08BDF9020004190FFA89F90FFA20
:103190008BFBD945DBDA1AEB0808BDF900004519AD
:1031A000D5E7BDE8F18F0000000402400038004080
:1031B000C8040020C6040020A004002080841E0053
:1031C0002DE9F04182B005000E0017009846089CDA
:1031D000A4B2009433009BB23A0092B2310089B29B
:1031E000280080B2FFF74AFFA4B2009443469BB286
:1031F0002A0092B2310089B2280080B2FFF73EFF68
:10320000A4B2009443469BB23A0092B2310089B214
:10321000380080B2FFF732FFA4B2009443469BB25D
:103220003A0092B2414689B2280080B2FFF726FFE9
:10323000BDE8F3812DE9F04182B005000E001700D2
:103240009846089CB6B21FFA88F846450DD2A4B23B
:10325000009433009BB23A0092B2310089B2280048
:1032600080B2FFF70BFF761CECE7BDE8F3812DE998
:10327000F44F82B004000D001E00BDF80800D0F12C
:1032800001075FF00108BDF808007FF0010101FBB4
:1032900000F95FF0000ABDF908B0320092B2BDF942
:1032A0000800411989B2200080B2FFF737FD3200D3
:1032B00092B2BDF90800291A89B2200080B2FFF746
:1032C0002DFD320092B2290089B2BDF90800001923
:1032D00080B2FFF723FD320092B2290089B2BDF916
:1032E0000800201A80B2FFF719FDB6B200962B0035
:1032F0009BB2BDF90800021992B2290089B2BDF94A
:103300000800201A80B2FFF7B9FE0FFA8AFA0FFA06
:103310008BFBDA454FDA3FB2002F05D4BBF1010B2E
:1033200019F1020919EB07071AF1010A18F102084D
:1033300018EB0707B6B200961BEB05039BB21AEB1E
:10334000040292B21BEB050189B2B4EB0A0080B211
:10335000FFF794FEB6B20096B5EB0B039BB2B4EB4D
:103360000A0292B2B5EB0B0189B21AEB040080B2EB
:10337000FFF784FEB6B200961AEB05039BB2B4EBDE
:103380000B0292B21AEB050189B21BEB040080B26A
:10339000FFF774FEB6B20096B5EB0A039BB2B4EB2E
:1033A0000B0292B2B5EB0A0189B21BEB040080B2AA
:1033B000FFF764FEA9E7BDE8F78F10B584B00400FD
:1033C00024B2642C01DB6420040024B25A2C09DBF3
:1033D0004FF4784000904523282236211020FFF733
:1033E00012FD07E0002000904523282236211020FE
:1033F000FFF709FD24B2502C09DB4FF47840009010
:103400005523282246211020FFF7FDFC07E000206D
:1034100000905523282246211020FFF7F4FC24B207
:10342000462C09DB4FF47840009065232822562172
:103430001020FFF7E8FC07E0002000906523282219
:1034400056211020FFF7DFFC24B23C2C09DB4FF69D
:10345000E43000907523282266211020FFF7D3FC6A
:1034600007E0002000907523282266211020FFF736
:10347000CAFC24B2322C09DB4FF6E43000908523DD
:10348000282276211020FFF7BEFC07E000200090E4
:103490008523282276211020FFF7B5FC24B2282CA2
:1034A00009DB4FF6E4300090952328228621102076
:1034B000FFF7A9FC07E00020009095232822862131
:1034C0001020FFF7A0FC24B21E2C09DB4FF4FC6097
:1034D0000090A523282296211020FFF794FC07E0F6
:1034E00000200090A523282296211020FFF78BFCB6
:1034F00024B2142C09DB4FF4FC600090B523282281
:10350000A6211020FFF77FFC07E000200090B523E4
:103510002822A6211020FFF776FC24B20A2C09DB12
:103520004FF4FC600090C5232822B6211020FFF73D
:103530006AFC07E000200090C5232822B621102055
:10354000FFF761FC24B2012C09DB4FF4FC60009012
:10355000D5232822C6211020FFF755FC07E00020C4
:103560000090D5232822C6211020FFF74CFC24B25E
:103570002200DFF8601902A801F040FB0020019052
:103580004FF6FF700090DFF8503902AA23210A207D
:10359000FFF7C6FC1FBD000040420F00A004002042
:1035A0007CB50400E4B2002C0BD0022C00F0C181E9
:1035B000C0F0E480042C00F00384C0F0C78200F067
:1035C00084BC47F6EF300090202340F23D120221E8
:1035D0000320FFF718FC4FF6E0700090022340F242
:1035E0003F1200210020FFF725FE4FF6E07000900B
:1035F000F023012200210020FFF71CFE4FF6E070AF
:103600000090202340F23F121E210020FFF712FEFF
:103610004FF6E0700090F02340F23F1220214FF46B
:103620009F70FFF707FE4FF6E0700090F02340F226
:103630003F12EE210020FFF7FDFD4FF6E0700090F5
:103640002023522200215020FFF7F4FD4FF6E070B6
:1036500000902023A2220021A020FFF7EBFD4FF6CF
:10366000E07000902023F2220021F020FFF7E2FD1D
:103670004FF6E0700090202340F23F1200214FF4FB
:103680009F70FFF7D7FD47F6EF3001904FF6FF70C0
:103690000090DFF84438DFF8302D08210320FFF7D1
:1036A0003FFC47F6EF3001904FF6FF700090DFF8D7
:1036B0002838DFF8182D08215320FFF731FC47F692
:1036C000EF3001904FF6FF700090DFF80C38DFF814
:1036D000002D0821A320FFF723FC47F6EF300190CF
:1036E0004FF6FF700090DFF8F037DFF8E82C082184
:1036F000F520FFF715FC4FF6E0700090EE2340F246
:103700003D1220214FF48770FFF75AFD4FF6E0700D
:1037100000903E2340F23D123E214FF48770FFF7A8
:10372000ADFC4FF6E07000905C2340F23D125C214E
:103730004FF48770FFF7A2FC4FF6E07000907A23F9
:1037400040F23D127A214FF48770FFF797FC4FF655
:10375000E0700090982340F23D1298214FF487705A
:10376000FFF78CFC4FF6E0700090B62340F23D125C
:10377000B6214FF48770FFF781FCA6E3002000908C
:10378000ED2340F20D1220210320FFF73CFB4FF404
:103790007840009020234F2202210220FFF74AFDAB
:1037A0004FF4784001904FF6FF700090DFF8283713
:1037B000DFF8142C08210320FFF7B2FB47F6EF30A7
:1037C0000090202340F23D120221F320FFF732FD4A
:1037D0004FF6E070009020234FF4A0721E21F020DD
:1037E000FFF728FD47F6EF3001904FF6FF7000908D
:1037F000DFF8E436DFF8DC2B0821F520FFF790FB3B
:103800004FF6FF70009035230F22D5212820FFF7B7
:10381000D7FC4FF6FF7000904523282245210F204A
:10382000FFF72CFC4FF6FF700090552328225521FE
:103830000F20FFF723FC4FF6FF700090652328222E
:1038400065210F20FFF71AFC4FF6FF7000907523DB
:10385000282275210F20FFF711FC4FF6FF70009012
:103860008523282285210F20FFF708FC4FF6FF70E3
:1038700000909523282295210F20FFF7FFFB4FF69C
:10388000FF700090A5232822A5210F20FFF7F6FB4B
:103890004FF6FF700090B5232822B5210F20FFF7C7
:1038A000EDFB4FF6FF700090C5232822C5210F20A5
:1038B000FFF7E4FB002001904FF6FF700090DFF867
:1038C0001836DFF8142BDA210A20FFF729FB002035
:1038D00001904FF6FF700090DFF8FC35DFF8FC2A0E
:1038E0003C214620FFF71CFB002001904FF6FF70A3
:1038F0000090DFF8E435DFF8E82A78214620FFF76A
:103900000FFB002001904FF4FC600090DFF8C835F9
:10391000C0A2462140F21D10FFF702FB00200090DC
:10392000EB2340F23B12B72140F21110FFF76BFA84
:10393000CBE200200090ED2340F20D122021032065
:10394000FFF761FA47F6EF30009020234F22022163
:103950000320FFF76FFC47F6EF3001904FF6FF7042
:103960000090DFF87435DFF8602A08210320FFF7A4
:10397000D7FA4FF6E0700090202352221E2100203B
:10398000FFF758FC4FF47840009020239F2202213B
:103990005320FFF74FFC4FF4784001904FF6FF7033
:1039A0000090DFF83435DFF8242A08215320FFF790
:1039B000B7FA4FF6E0700090DC234FF482722821B2
:1039C0000A20FFF7FDFB3A200500ADB2DC2D0CDA32
:1039D0004FF6E07000902B009BB23C22290089B288
:1039E0000A20FFF74BFB1235EFE74FF6E07000902F
:1039F000DC233C2228213C20FFF740FB3C20050033
:103A0000ADB2B5F5827F10DA3A200600B6B2DC2EF0
:103A100009DA4FF6E072310089B2280080B2FFF770
:103A20007DF91236F2E71435EAE7002001904FF6EF
:103A3000FF700090DFF8A434D6A2B9214FF4917042
:103A4000FFF76EFA002001904FF6FF700090DFF84C
:103A50008834D1A232211E20FFF762FA00200190A3
:103A60004FF6FF700090DFF87034CCA257211E2073
:103A7000FFF756FA002001904FF6FF700090DFF834
:103A80005834C7A27A211E20FFF74AFA002001907D
:103A90004FF6FF700090DFF84034C2A2A0211E2034
:103AA000FFF73EFA002001904FF6FF700090DFF81C
:103AB0002834BDA2C3211E20FFF732FA0020019056
:103AC0004FF6FF700090DFF81434B8A2E2213B20DB
:103AD000FFF726FA002001904FF6FF700090DFF804
:103AE000FC33B3A2E2216120FFF71AFA0020019013
:103AF0004FF6FF700090DFF8E433AEA2E221892098
:103B0000FFF70EFA002001904FF6FF700090DFF8EB
:103B1000CC33A9A2E221B120FFF702FA00200190E4
:103B20004FF6FF700090DFF8B433A4A2E221D92051
:103B3000FFF7F6F9002001904FF6FF700090E74B79
:103B4000E2A2E221FA20FFF7EBF9BEE100200090AB
:103B5000ED2340F20D1220210320FFF754F947F620
:103B6000EF30009020239F2202215320FFF762FBB9
:103B700047F6EF3001904FF6FF700090D64BDFF81C
:103B80004C2808215320FFF7CBF94FF6E070009046
:103B90002023A0221E215220FFF74CFB4FF4784037
:103BA00000902023EF220221A320FFF743FB4FF4D4
:103BB000784001904FF6FF700090C74BDFF8102857
:103BC0000821A320FFF7ACF900200090EB2340F27E
:103BD0003B12B72140F21110FFF715F94FF6E070D4
:103BE0000090DC234FF4827228210A20FFF7E8FAC4
:103BF0003A200500ADB2DC2D0EDA4FF6E0700090F1
:103C00002B009BB23C22290089B20A20FFF736FA2A
:103C10001235EFE7435600004FF6E0700090DC23CA
:103C20003C2228213C20FFF729FA3C200500ADB2B8
:103C3000B5F5827F10DA3A200600B6B2DC2E09DA3A
:103C40004FF6E072310089B2280080B2FFF766F8C3
:103C50001236F2E71435EAE7002001904FF6FF70C4
:103C600000909E4B4BA2B9214FF49170FFF758F989
:103C7000002001904FF6FF700090984B94A2D42141
:103C80004FF49170FFF74CF9002001901F20009035
:103C9000924BDFF85027DE2140F21110FFF740F978
:103CA000002001904FF6FF7000908B4B3AA232211A
:103CB0001E20FFF735F9002001904FF6FF700090AD
:103CC000854B36A257211E20FFF72AF900200190CC
:103CD0004FF6FF700090804B31A27A211E20FFF733
:103CE0001FF9002001904FF6FF7000907A4B2DA233
:103CF000A0211E20FFF714F9002001904FF6FF705D
:103D00000090754B28A2C3211E20FFF709F900205F
:103D100001904FF6FF700090704B24A2E2213B20EF
:103D2000FFF7FEF8002001904FF6FF7000906B4BFC
:103D30001FA2E2216120FFF7F3F8002001904FF667
:103D4000FF700090654B1BA2E2218920FFF7E8F885
:103D5000002001904FF6FF700090604B16A2E22108
:103D6000B120FFF7DDF8002001904FF6FF700090C2
:103D70005A4B12A2E221D920FFF7D2F8002001907D
:103D80004FF6FF700090554B50A2E221FA20FFF74A
:103D9000C7F89AE06D4100003900000037000000CC
:103DA000350000003300000031000000300000004A
:103DB000320000003400000036000000380000002F
:103DC00000200090ED2340F20D1220210320FFF788
:103DD0001AF847F6EF3000902023EF220221A320AB
:103DE000FFF728FA47F6EF3001904FF6FF7000908A
:103DF000394BDFF8DC250821A320FFF791F84FF6B7
:103E0000E07000902023F0221E21A220FFF712FA7A
:103E10004FF478400090202340F23D120221F3201D
:103E2000FFF708FA4FF4784001904FF6FF700090CA
:103E3000294BDFF8A0250821F520FFF771F80020B5
:103E400001904FF6FF700090234BDFF89C253C213A
:103E50001420FFF765F8002001904FF6FF700090E6
:103E60001D4BDFF8882550211420FFF759F800205A
:103E700001904FF6FF700090174BDFF87425642116
:103E80001420FFF74DF8002001904FF6FF700090CE
:103E9000114BDFF8602578211420FFF741F800204E
:103EA00001904FF6FF7000900B4BDFF84C258C21F2
:103EB0001420FFF735F800200090EB2340F23B126E
:103EC000B72140F21110FEF79EFF73BD31300000A4
:103ED0006D560000A4A4000804010020FC0000208E
:103EE00070B582B004000D00EDB2012D03D14FF486
:103EF000FC60060002E04FF478400600E4B2012CBA
:103F000027D1B6B200968E2340F22712852140F2C7
:103F10001F10FEF778FFB6B200967E2340F22F12F4
:103F2000852140F22710FFF7A9F8B6B20096942336
:103F300040F22F128E2140F22710FFF79FF8B6B201
:103F40000096942340F22F127E2140F22F10FFF7AB
:103F500095F8E4B2022C2FD133009BB20A22A6219D
:103F60004FF49470FFF783F900200090B42340F2DF
:103F70003312A6214FF48F70FEF745FFB6B20096BC
:103F8000AE234FF49172A6214FF49270FFF776F8AA
:103F9000B6B20096AE234FF49472A6214FF49470FB
:103FA000FFF76CF8B6B20096AE234FF49772A621D5
:103FB0004FF49670FFF762F873BD2DE9FD4F82B0A4
:103FC0000D000E9C00275FF000089DF808000128F6
:103FD0002CD0022854D1DFF824040078BD280EDA52
:103FE000DFF818040078DFF8181421F81050DFF813
:103FF0000C040078401CDFF80414087015E0002061
:104000000600B6B2BD2E0CDAB6B2DFF8F40310EB40
:1040100046004088B6B2DFF8E81321F81600761C97
:10402000EFE7DFF8DC03A0F87A5129E0DFF8D403EA
:104030000088BD280EDADFF8CC030088DFF8C8134B
:1040400021F81050DFF8BC030088401CDFF8B413DF
:10405000088015E000200600B6B2BD2E0CDAB6B21C
:10406000DFF8A40310EB46004088B6B2DFF89813DF
:1040700021F81600761CEFE7DFF88C03A0F87A51E0
:104080009DF80C00012840F09C813D200600B6B24E
:10409000FB2E80F27F81E4B2002C1DD11FFA88F83C
:1040A000D74830F81800B22148430A2190FBF1F0BC
:1040B0000A2190FBF1F082461FFA88F8D04810EBF5
:1040C00048004088B22148430A2190FBF1F00A21C0
:1040D00090FBF1F0834665E0E4B2012C1DD11FFA9C
:1040E00088F8C74830F81800B2214843642190FB93
:1040F000F1F00A2190FBF1F082461FFA88F8C048DF
:1041000010EB48004088B2214843642190FBF1F055
:104110000A2190FBF1F0834644E0E4B2022C1FD167
:104120001FFA88F8B64830F81800B22148434FF417
:104130007A7190FBF1F00A2190FBF1F082461FFAB0
:1041400088F8AF4810EB48004088B22148434FF44C
:104150007A7190FBF1F00A2190FBF1F0834621E0A7
:10416000E4B2032C1ED11FFA88F8A54830F81800D5
:10417000B221484342F2107190FBF1F00A2190FB0A
:10418000F1F082461FFA88F89D4810EB48004088FD
:10419000B221484342F2107190FBF1F00A2190FBEA
:1041A000F1F08346BAF1B30F01D3B0208246BBF1E0
:1041B000B30F01D3B0208346B6B2502E17D0B6B29B
:1041C000632E14D0B6B2762E11D0B6B2892E0ED090
:1041D000B6B29C2E0BD0B6B2AF2E08D0B6B2C22E5D
:1041E00005D0B6B2D52E02D0B6B2E82E00D17F1CD3
:1041F000BAF1000F59D081480078BD280ADB0020B1
:104200000090DB23B819421C92B22921B81980B260
:10421000FEF7F9FDDA4536D0DA4517D2BBEB0A00D6
:1042200081464FF47842DBF1DB005FFA89F919EB44
:10423000000189B2B81980B2FEF770FDB9F1010929
:104240005FFA89F9B9F1000FEBD12EE0D3452CD2FA
:10425000BBF1000F29D0BAEB0B0081464FF4784236
:10426000DBF1DB005FFA89F9B0EB090189B2B8191B
:1042700080B2FEF753FDB9F101095FFA89F9B9F18E
:10428000000FEBD111E04FF47842DAF1DB0189B293
:10429000B81980B2FEF742FD4FF47842DAF1DA0144
:1042A00089B2B81980B2FEF739FD9DF810000128D7
:1042B0006CD11FFA88F8544830F81800B2214843EE
:1042C00042F2107190FBF1F082461FFA88F84E48D6
:1042D00010EB48004088B221484342F2107190FB35
:1042E000F1F08346BAF1B30F01D3B0208246BBF19F
:1042F000B30F01D3B0208346BAF1000F46D0DA45A0
:1043000034D0DA4516D2BBEB0A0081461F22DBF11E
:10431000DB005FFA89F919EB000189B2B81980B2A4
:10432000FEF7FCFCB9F101095FFA89F9B9F1000F58
:10433000ECD12BE0D34529D2BBF1000F26D0BAEB4C
:104340000B0081461F22DBF1DB005FFA89F9B0EB3D
:10435000090189B2B81980B2FEF7E0FCB9F1010990
:104360005FFA89F9B9F1000FECD10FE01F22DAF101
:10437000DB0189B2B81980B2FEF7D0FC1F22DAF156
:10438000DA0189B2B81980B2FEF7C8FC18F1010849
:10439000761C7CE63C200600B6B2B6F5827F10DAC9
:1043A0003A200700BFB2DC2F09DA4FF6E07239007D
:1043B00089B2300080B2FEF7B1FC1237F2E7143652
:1043C000EAE705B0BDE8F08FACA40008B4A400088B
:1043D000BCA40008C4A40008CCA40008D4A400080D
:1043E000DCA40008E4A40008C4A30008D4A30008C7
:1043F000E4A30008ECA4000838A40008E1040020AD
:1044000024010020CA040020A002002010B51021C1
:10441000DFF88C04FEF7F3F8D72001F050F901F033
:1044200065F904002006FAD51021DFF87404FEF7C0
:10443000E4F810BD10B586B003A8DFF868141CC9F5
:104440001CC00C390C3801F0D1F81021DFF85004F1
:10445000FEF7D3F802A800F036F802229DF8081003
:1044600003A8FDF7C1FA02229DF809100DF10F0013
:10447000FDF7BAFA02229DF80A100DF11200FDF7BD
:10448000B3FA02229DF80B100DF11500FDF7ACFAFE
:10449000002001904FF6FF700090DFF80C34DFF839
:1044A0000C2446210A20FEF73BFD002001904FF628
:1044B000FF700090DFF8F03303AA4621B420FEF726
:1044C0002FFD06B010BD38B50400FFF79FFF102187
:1044D000DFF8CC03FEF793F89F2001F0F0F80020FE
:1044E0000500EDB2042D05DA01F000F9EDB2285512
:1044F0006D1CF6E71021DFF8A803FEF77EF831BD4A
:104500002DE9F04104000D0016001F005FF00008C7
:10451000FFF77CFF1021DFF88803FEF770F8E4B2A4
:10452000012C03D1842001F0CAF807E0E4B2022C88
:1045300003D1872001F0C3F800E01DE0002001F066
:10454000BEF8002001F0BBF82800C0B280B201F034
:10455000B6F8002080461FFA88F8B6B2B04507D2F8
:10456000387880B201F0ABF87F1C18F10108F2E74F
:104570001021CB48FEF741F8BDE8F08138B50400C2
:104580000D00FFF743FF1021C548FEF738F8E4B2ED
:10459000012C03D1832001F092F807E0E4B2022C51
:1045A00003D1862001F08BF800E016E02800C0B2AD
:1045B000C009C0B280B201F082F82800C0B2400049
:1045C00080B201F07CF8002001F079F81021B448A5
:1045D000FEF713F82820FEF79FF831BD38B5040028
:1045E0000D00FFF713FF1021AD48FEF708F8E4B205
:1045F000012C03D1532001F062F807E0E4B2022C51
:1046000003D1552001F05BF800E016E02800C0B2AD
:10461000C009C0B280B201F052F82800C0B2400018
:1046200080B201F04CF8002001F049F810219C48BC
:10463000FDF7E3FF2820FEF76FF831BD2DE9F041CB
:1046400004000D0016001F005FF00008FFF7DEFEFB
:1046500010219348FDF7D3FFE4B2012C03D1D420FD
:1046600001F02DF807E0E4B2022C03D1D62001F0CE
:1046700026F800E01FE0FF2001F021F8002001F003
:104680001EF82800C0B280B201F019F8FF2001F036
:1046900016F8002080461FFA88F8B6B2B04506D258
:1046A00001F024F838707F1C18F10108F3E710219D
:1046B0007B48FDF7A2FFBDE8F081FEB504000D00C8
:1046C0001600E4B22000012802D002287CD0E2E0EB
:1046D000F6B2012E07D076D3032E22D012D3052EA8
:1046E00050D02DD36FE001210220FFF777FF00AB00
:1046F000012200210220FFF7A1FF00A801F010F81D
:10470000070060E002210220FFF768FF00AB0122F2
:1047100000210220FFF792FF00A801F001F8070036
:1047200051E003210220FFF759FF00AB01220021D5
:104730000220FFF783FF00A800F0F2FF070042E02D
:1047400004210220FFF74AFF01AB062200210220CC
:10475000FFF774FF01A800F0E7FF00F0DDFA54490D
:10476000086053480068534900F05AFC05D9504886
:104770000068002100F0DCFF03D84D485FF07E5157
:10478000016020E005210220FFF728FF01AB06228F
:1047900000210220FFF752FF01A800F0C5FF00F042
:1047A000BBFA4549086044480068424900F038FCBB
:1047B00005D941480068002100F0BAFF03D83E48FF
:1047C0005FF07E51016066E0F6B2012E07D062D341
:1047D000032E26D014D3052E49D033D35BE0ADB2DF
:1047E0002A002EA100A800F009FA00AB0122002146
:1047F0000120FFF785FE01210120FFF7BFFE4AE0FF
:10480000ADB22A0025A100A800F0F8F900AB012202
:1048100000210120FFF774FE02210120FFF7AEFE08
:1048200039E0ADB22A001DA100A800F0E7F900AB05
:10483000012200210120FFF763FE03210120FFF781
:104840009DFE28E01A48006800F0B0F902000B0055
:104850001A4901A800F0D2F901AB0622002101207B
:10486000FFF74EFE04210120FFF788FE13E01248F7
:10487000006800F09BF902000B00104901A800F04D
:10488000BDF901AB062200210120FFF739FE052109
:104890000120FFF773FE380080B2FEBD25640000E2
:1048A0000000024044A4000804010020F4A3000812
:1048B000140100200100204118010020F4A4000888
:1048C00070B504000D00290089B2200000F0BDF889
:1048D000290089B2200000F0B0F8002801D10220A0
:1048E0002BE0290089B2200000F0BDF8290089B230
:1048F000200000F099F84FF4F070FDF719FF29003F
:1049000089B2200000F087F8290089B2200000F069
:104910009CF83C20FDF70CFF290089B2200000F034
:104920008CF8002802D10020060001E001200600DA
:104930004FF4AF70FDF7FCFE300070BDF8B5040019
:104940000D00160000200700FFB2082F0AD0320029
:1049500092B229000120B8402040C0B200F003F814
:104960007F1CF1E7F1BD70B504000D0016003100A9
:1049700089B2280000F077F8310089B2280000F0F1
:1049800053F8E4B2002C0BD13C20FDF7D1FE3100EE
:1049900089B2280000F03FF80420FDF7C9FE0AE0C4
:1049A0000420FDF7C5FE310089B2280000F033F87D
:1049B0003C20FDF7BDFE310089B2280000F045F82B
:1049C00070BD70B504000D00290089B2200000F010
:1049D0004AF8290089B2200000F026F80120FDF7EE
:1049E000A7FE290089B2200000F02FF80420FDF76F
:1049F0009FFE290089B2200000F01FF8002802D095
:104A00000120060001E0002006003C20FDF790FE9A
:104A10003000C0B270BD38B504000D00290089B265
:104A20002000FDF7EAFD31BD38B504000D00290076
:104A300089B22000FDF7E3FD31BD0200108A084273
:104A400001D0012000E00020704738B504000D00BF
:104A50000D48ADB205600C48002101710A492000E3
:104A6000FDF76AFD31BD38B504000D000648ADB252
:104A70000560054801210171034800218171024947
:104A80002000FDF759FD31BD780400202DE9F44FD9
:104A900084B004000D001E00002001900020834619
:104AA000290089B22000FFF70BFF8DF800009DF868
:104AB0000000002802D09DF8000074E02A0092B2A5
:104AC0002100F020FFF73AFF0020029001200700AC
:104AD000002082465FFA8AFABAF1080F57D05FFACF
:104AE0008AFA5FFA8BFB16EBCB0000210AF8001064
:104AF000002081465FFA89F9B9F1080F44D02900F6
:104B000089B22000FFF75DFF8046290089B22000AE
:104B1000FFF757FF8DF801005FFA88F8B8F1000F32
:104B20000FD19DF8010000280BD10198074202D057
:104B30000120804604E00198791E08403843029025
:104B40007F002A0092B221004046C0B2FFF70BFF5F
:104B50005FFA88F8B8F1000F13D05FFA8AFA5FFAAB
:104B60008BFB16EBCB005FFA8AFA5FFA8BFB16EB36
:104B7000CB011AF80110012212FA09F211430AF8C6
:104B8000001019F10109B5E71AF1010AA2E702982C
:104B900001901BF1010B019800287FF481AF04986C
:104BA00080F800B0002005B0BDE8F08F5FF0FF0C8A
:104BB0001CEAD05114BF614506E0C110400721F046
:104BC000E04101F16051704779B900F00041000205
:104BD0000AD0B0FA80FC00FA0CF001F16051A1EBB0
:104BE0000C5101EBD0214005704741020CBF40F44D
:104BF000E0016FF000010020704700000CB41CB50C
:104C0000044604A801900A46009401AB00A9074895
:104C10007844183000F09EFD009900220A700028A8
:104C20005CBF0098001B16BC5DF80CFB03D9FFFFAE
:104C300070B44FF0004591EA030C44BF6B4001F0A3
:104C4000F7BD00BF841A71EB030603D2001BB1410C
:104C5000121973414FF4001C1CEB410F34BF7CEB65
:104C6000430443E00C0DA4EB1356352E50DC45EA0B
:104C7000C323DB0A45EAC121C912B6F120050DDDC7
:104C800063FA05F6EB4086EA0305124218BF45F0C9
:104C90000105C01851F100010CD213E062FA06F5CB
:104CA000F2405540F3415A40B340F3405A40801817
:104CB000594107D349085FEA30005FEA350528BF4C
:104CC00045F0010501F58011420875F1004250F1EF
:104CD000000041EB045170BC4FF4001C1CEB410F71
:104CE00038BF70470020090D090570471CEB410FC4
:104CF00010D252EA43060BD0BCEB410F05D80C0D85
:104D0000AB43661E342EB5DD02E0AB43801859413B
:104D100070BC704770BC70474FEAF17CBCF1E04C4E
:104D20002CBFBCF5001F11E05FEA4C0C34BFBCF196
:104D30007F5F2EE05FEA9C0C4FEA0C1C4FEA3C0CB4
:104D4000C10071F100414CEB50707047C90241EA5B
:104D50005051C00218BF41F0010141F000414FEA3B
:104D60006C50C0F10900212810D240EACC7CCCF173
:104D7000200C11FA0CF070F10040CCF1200C21FA5B
:104D80000CF00CF0004C40EB0C0070474FEACC707C
:104D90007047490011F5001F04D84FEACC10FF30CE
:104DA000C0057047C8177047F0B540F2FF7581EA3B
:104DB000030C0CF0004C15EA11541DBF15EA1357F3
:104DC000AC42AF42E5E0BC41C1F31301C3F31303AE
:104DD000801A994143F4801304D2641E4000494173
:104DE00080185941C90241EA5051B1FBF3F603FB67
:104DF0001611A2FB0675D7EBC020A94102D2761E80
:104E000080185941C90241EA5051B1FBF3FE03FB3E
:104E10001E11A2FB0E75D7EBC020A94103D2AEF143
:104E2000010E80185941890241EA9051760546EAFF
:104E30008E2EB1FBF3F603FB1611A2FB0675D7EB22
:104E40008020A94102D2761E80185941C90241EA48
:104E500050514EEA060EB1FBF3F603FB1611A2FB0E
:104E60000675D7EBC020A94102D2761E80185941A1
:104E7000C90241EA5051B1FBF3F703FB1711A2FB42
:104E80000735D3EBC020A94167F100070CBF0042F2
:104E900047F0010766F3D5274FEA1E31B80814F52D
:104EA000806412DDBD0775F1004250EB0E5051EBEE
:104EB000045111F5801F5CBF41EA0C01F0BD4CF0BC
:104EC0007F6141F0E0410020F0BDBD076D0840EA80
:104ED0000E5041F48011D4F10104B4F120060ADA35
:104EE000C4F120060200E04001FA06F3E140184355
:104EF000B24015430EE0342C13DCC6F1200445EA21
:104F000040056D0820FA06F2154321FA06F0A1408B
:104F10000D43002175F1004250F1000051EB0C01EE
:104F2000F0BD00205FEA0C01F0BDCFB992185B41E3
:104F3000B3FA83F704BFB2FA82F6BF190B3FB7F199
:104F400020062FBF02FA06F3BB40C7F1200622FA63
:104F500006F638BF3343BA401CB1E419641E33E788
:104F60007F4231F00041B1FA81F404BFB0FA80F61B
:104F7000A4190B3CB4F120062FBF00FA06F1A140A2
:104F8000C4F1200620FA06F638BF3143A0403C1B8E
:104F90001AE7AC421ABF05EA1357AF4212E050EAD3
:104FA00041061CBF52EA4306BFE750EA41073046BC
:104FB00061461CBF41EA0551F0BD52EA430C08BFEF
:104FC000C143F0BD00204FF4001616EB410F98BF0F
:104FD00016EB430F08BF16EB410F24BFC14305E09A
:104FE00016EB430F0CBF61464CEA0551F0BD0000C3
:104FF0004FF4001C1CEB410F94BF1CEB430F09E066
:1050000041EA030C50EA4C0C52EA0C0C03D28B42DE
:1050100008BF8242704714BF994290427047000017
:105020004FF0807C1CEB400F94BF1CEB410F05E060
:1050300040EA010C5FEA4C0C01D28142704718BF74
:1050400088427047002800BF0AD0B0FA80F188403B
:10505000D1F19D01C905020672F1004241EB102019
:1050600070470000FF2212EAD05C1DBF12EAD15344
:10507000944593422BE09C44D30780EA01021A40F6
:1050800043EA002043EA0121A1FB0030410038BF80
:1050900040007CF17F010BDBFE294ADA5B0842EA23
:1050A000C15153EA006373F1004C51EB102070477B
:1050B000D1F1080CDCF120012FDB5B0810FA01F1C3
:1050C0000B4373F1004120FA0CF0504170479445B6
:1050D0001CBF02EAD153934280EA010202F000426F
:1050E0001DD0400019D0490017D05BB9634514D0DA
:1050F0000902B1FA81F39940BCEB030CC00140F006
:105100000040C1E70002B0FA80FC10FA0CF0B3EBEB
:105110000C0CC90141F00041B6E710007047400097
:105120000AD0490008D010F1807F94BF11F1807F30
:1051300002E042F0FF407047D0437047B0B581EACB
:10514000030C0CF0004C40F2FF7515EA11541DBF22
:1051500015EA1357AC42AF4239E0E41923EA45534C
:1051600043F48013C90241F0004141EA505EC70296
:105170001100A7FB020200284FF00000EEFB012007
:105180004FF00001E3FB072118BF42F00102401875
:1051900000214941E3FB0E01A4F580640F0302D214
:1051A00052004041494154F101046CDD470872F15D
:1051B000004250F1000051EB0451A1F580115CBF99
:1051C00041EA0C01B0BD4CEA05510020B0BD05EA32
:1051D0001357AC4214BFAF4241E050EA410E1CBF2E
:1051E00052EA430E02E061460020B0BD24423C4436
:1051F0001BD15FEA070EF6D0090302BF014600206B
:10520000AEF1140EB1FA81F7AEEB070401FA07FE16
:105210000C37C7F1200100FA07F7C8404EEA000E2C
:1052200023EA455343F48013A2E733F00043B3FA73
:1052300083F704BFB2FA82FE77440B3FE41BB7F159
:10524000200E2FBF02FA0EF3BB40C7F1200E22FA48
:105250000EFE38BF43EA0E03BA40641C82E750EAF0
:10526000410E14BF52EA430E6FF000014FF40017D5
:1052700017EB430F8ABF194617EB410FB5E74CEA0E
:1052800005510020B0BDD4F10104B4F120070FDABC
:10529000C4F12007520828BF42F0010210FA07F5B6
:1052A00001FA07F7E1BF2A43E0403843E1400FE04D
:1052B000352C98DCC7F1200452EA400220FA07F2AC
:1052C00018BF42F0010231FA07F0A1400A43002161
:1052D00072F1004250F1000051EB0C01B0BD000032
:1052E0004100090E7F3915D4D1F11F0114D44000BB
:1052F00007D2C00140F00040C84048BF6FF00040F6
:105300007047C00140F00040C8404CBF4FF0004023
:10531000404270470020704700424FF0004058BFA5
:10532000C0437047010040F10980F446404200F05C
:1053300005F851F000416047010000BF09D0B0FA04
:1053400080F18840C91CC1F58461090501EBD021B9
:1053500040057047F446400D40EAC120490006D29E
:1053600000F014F8004248BF6FF00040604700F0C2
:105370000DF84FF0004188428CBF0846404260471C
:10538000400D40EAC120490080F00D8040F000400F
:10539000490DA1F58061491C05D4D1F11F0154BF0D
:1053A000C840C01770474FF000007047DFF8A810E2
:1053B000C0B208607047C9B2002905D0284A1268F7
:1053C0000243274B1A6004E0254A12688243244BAB
:1053D0001A607047C9B2002905D0224A12680243F8
:1053E000204B1A6004E01F4A126882431D4B1A606A
:1053F0007047C9B2002905D01B4A126802431A4BF4
:105400001A6004E0184A12688243174B1A6070470A
:1054100010B40100002200230020C9B24C09E4B2FC
:105420002200012A03D10B4C2468230002E00B4C1C
:1054300024682300C9B211F01F04220033FA02F4D9
:10544000E40702D50124200001E000242000C0B2BE
:1054500010BC704700380240000047423438024018
:105460001C380240203802402438024030B4002268
:105470000F2311F00304E4B2A400A3401A00C9B240
:105480008B100E4C54F823309343C9B28C100B4D43
:1054900045F82430C9B28B10084C54F82330C0B200
:1054A00011F00304E4B2A40010FA04F42343C9B2D7
:1054B0008C10024D45F8243030BC70470800014084
:1054C000F0B4002300210F22C478002C21D0174C07
:1054D000246814F4E064D4F5E064240A2300D3F1D2
:1054E00004042100D2B21A4144788C40230084780D
:1054F000144023431B0104780D4D63550478641157
:105500000C4D0126077817F01F07BE4045F82460B0
:1055100009E004786411084D0126077817F01F0789
:10552000BE4045F82460F0BC704700000CED00E080
:1055300000E400E000E100E080E100E010B40022BF
:1055400003881A0012F441520B884C8823438C883C
:105550002343CC8823430C8923434C8923438C89E0
:105560002343CC8923431A430280838B4FF2FF7479
:10557000234083830B8A038210BC7047C9B2002981
:1055800004D0028852F04002028004E002884FF604
:10559000BF731A40028070478089704781817047CD
:1055A0000200002013890B4202D00123180001E001
:1055B00000231800C0B2704738B504000D00EDB2EA
:1055C000A58102212000FFF7EBFF0028F9D001217F
:1055D0002000FFF7E5FF0028F9D080212000FFF729
:1055E000DFFF0028F9D1A089C0B232BD00B587B075
:1055F00001210120FFF7DFFEE020009002208DF85E
:10560000040003208DF8050000208DF8060000201E
:105610008DF8070000A94048FCF78EFF0522052100
:105620003D48FCF7EEFF052206213B48FCF7E9FF69
:10563000052207213848FCF7E4FF102000900120E4
:105640008DF8040003208DF8050000208DF8060079
:1056500001208DF8070000A92F48FCF76DFF0121FC
:105660004FF48050FFF7B6FE00212C48FFF786FF6D
:105670000020ADF808004FF48270ADF80A00002059
:10568000ADF80C000220ADF80E000120ADF81000BE
:105690004FF40070ADF812000020ADF814000020A7
:1056A000ADF816000720ADF8180002A91B48FFF757
:1056B00045FF01211948FFF761FF07B000BD10B594
:1056C000040002211548FFF76BFF0028F9D02100E4
:1056D00089B21248FFF762FF01211048FFF760FF0F
:1056E0000028F9D00D48FFF757FF10BD80B5022103
:1056F0000A48FFF755FF0028F9D000210748FFF7B7
:105700004DFF01210548FFF74BFF0028F9D0034862
:10571000FFF742FF02BD00000000024000300140E0
:105720000A22002101F0C6B90022002101F08ABA44
:105730004FF0807C1CEB400F94BF1CEB410F05E049
:1057400040EA010C5FEA4C0C01D28842704718BF56
:10575000814270472DE9F04F80460FF2B450A5B05A
:1057600017461D46D0E90023CDE9122304AE0020E0
:105770000491706214AC00E04F440020ADF80200C8
:1057800012AB4FF0FF3239460DF1020001F05CFA26
:105790008146B9F1010F08DA3878B0F1010969EBF7
:1057A00009096FEA09004FEAD079BDF802002528FF
:1057B0000CBFA9F101034B46012B07DB3A4602A9B6
:1057C000404601F005F8002800F19D82BDF8020076
:1057D000252807D10020F06030617061B061F06170
:1057E000306205E00028C7D1706A8EE240F0010007
:1057F00017F8011F2029F9D023290DD02B2904D017
:105800002D2906D030290AD00CE040F0020080B2E9
:10581000EEE740F00400FAE740F00800F7E740F058
:105820001000F4E72A290DD129680A1D2A600968A9
:10583000F162002904D5494240F00400F16280B2CF
:105840007F1C13E00021F1620BE0F16A6FF000436E
:10585000994205D001EB810302EB43013039F1623B
:105860007F1C3A78A2F130010A29EED339782E292B
:1058700003D04FF0FF31B1621EE017F8011F2A2953
:1058800006D129680A1D2A607F1C0968B16213E0ED
:105890000021B1620BE0B16A6FF00043994205D07C
:1058A00001EB810302EB43013039B1627F1C3A788E
:1058B000A2F130010A29EED330860FF25C4039782C
:1058C00001F0D2F908B117F8010B8DF842009DF8EC
:1058D0004200682802BF39786829622005D06C2808
:1058E00004BF38786C2803D171208DF842007F1CEA
:1058F00014A8B0603978B1F1250025D01C387BD0D0
:10590000001F022878D9133800F0A080093873D01E
:10591000801E00F03181401E00F0DB80401E022816
:105920006AD9001F00F0D580401F3AD0401E00F019
:105930008D80401E2AD0C01E0BD0801E00F08680B5
:10594000C01E00F0838037E1F068411CF160252122
:105950003BE19DF842006C28286813D0011D2960A6
:105960000068B26A7060002A02D501F089F907E088
:10597000002101F0A1F900281ABF7168401AB06A2D
:10598000306123E1011D296002680EE12868011DD4
:10599000296000210068CDE9020114A87060782117
:1059A000E6E09DF84200622818D0682806D06A28F0
:1059B0000BD06C2819D0712807D016E02868011D7B
:1059C00029600068716A018000E12A68101D286062
:1059D0001268706AC117C2E90001F7E02868011D6A
:1059E00029600068716A0170F0E02868011D296073
:1059F0000068716A0160E9E02868C01D20F00700B6
:105A0000286000F108022A60D0E90023CDE90223D2
:105A1000002B04D5F068421CF2602D220DE0308E80
:105A2000820704D5F068421CF2602B2205E0C00713
:105A300004D5F068421CF26020220255F06814AAD6
:105A40008018706002A800F0BBFBBFE09DF8420028
:105A50006C2808BF2A6811D0712808BF2A6802D0B4
:105A60002A686A280AD1D21D22F007022A609446C9
:105A70000CF108022A60DCE9002303E0131D2B600F
:105A800000231268CDE90223682808BF92B207D02C
:105A9000622808BFD2B203D0742818BF7A2802D176
:105AA0000023CDE9022396F8300000075CD5DDE93C
:105AB0000223002B08BF002A56D041F0200078288E
:105AC00052D1F06830220255401C421CF260015550
:105AD0004AE09DF8420062280CD0682810D06A285D
:105AE0001AD06C2823D0712816D074281FD07A2899
:105AF0000CD01CE02868021D2A6090F900201AE0F2
:105B00002868021D2A60B0F9002014E02868021DF0
:105B10002A60002302680FE02868C01D20F00700FB
:105B2000286000F108022A60D0E9002304E0286818
:105B3000021D2A600268D317CDE90223002B04DA84
:105B4000F068421CF2602D220DE0308E820704D5F1
:105B5000F068421CF2602B2205E0C00704D5F06813
:105B6000421CF26020220255F06814AA801870606E
:105B700002A800F076FA29E09DF842006C2807D0D0
:105B8000F068411CF16029680A1D2A6009681CE060
:105B90002868011D296001AA0068ADF804000020F2
:105BA000ADF806004FF0FF30B06202A9404600F0A9
:105BB000B7F800280AD5A6E0F068421CF26025225A
:105BC000025519B1F068421CF2600155F06AF168A3
:105BD000401AB169401A3169401AF169401A716975
:105BE000401A316AA0EB010996F830007F1C40078B
:105BF00011D420208DF800004FF0000A09E00123A5
:105C000000AA02A9404600F0E3FD00287BD10AF17A
:105C1000010ACA45F3DBF36814AA02A9404600F062
:105C2000D7FD00286FD13020D6F818A08DF80000DD
:105C30004FF0000B09E0012300AA02A9404600F042
:105C4000C7FD00285FD10BF1010BD345F3DB3369AE
:105C5000726802A9404600F0BBFD002853D13020F5
:105C6000D6F81CA08DF800004FF0000B09E00123CE
:105C700000AA02A9404600F0ABFD002843D10BF179
:105C8000010BD345F3DB30697168D6F814A000EB43
:105C9000010B0AE01BF8011B0498C047049090B365
:105CA000706A401C7062AAF1010ABAF1000FF1D1CA
:105CB0003020D6F820A08DF800004FF0000B08E04F
:105CC000012300AA02A9404600F082FDD8B90BF1D9
:105CD000010BD345F4DB96F8300040077FF54DAD5E
:105CE00020208DF800004FF0000A01E00AF1010ABF
:105CF000CA45BFF642AD012300AA02A9404600F002
:105D000067FD0028F2D04FF0FF3025B0BDE8F08FDE
:105D10000000000000000000686A6C747A4C00000B
:105D20002DE9F04F0F4695B03C6B83469146002C11
:105D300048BF6FF0004400F0EBFF796B4018029011
:105D40000FF6BC22D2E90001CDE9030197F8380033
:105D5000400702D40298412805D240200DF1140AD0
:105D60000290002509E000F0D9FF5FEA000AF8D1AF
:105D70004FF0FF3072E1A4EB0804012CC0F2B580B3
:105D8000B9F8001003AA0DF1010001F01FF88046D8
:105D9000002800F1C180B9F8000018B9B8F1010875
:105DA00000F1BA804445C0F2A0807869029908EBFE
:105DB0000002914280F08A807D634042396A401A35
:105DC000B969401A796A401AF969401AB96A451ADC
:105DD00097F83800400710D420208DF800000026E6
:105DE00009E0012300AA3946584600F0F1FC0028DA
:105DF00040F09280761CAE42F3DB7B695246394616
:105E0000584600F0E5FC002840F0868030208DF8F0
:105E100000000026386A019008E0012300AA3946F4
:105E2000584600F0D5FC002876D1761C01988642B1
:105E3000F3DBBB69FA683946584600F0C9FC002814
:105E40006AD130208DF800000026786A019008E0C1
:105E5000012300AA3946584600F0BAFC00285BD15D
:105E6000761C01988642F3DBB869F968FB69421831
:105E70003946584600F0ACFC00284DD130208DF852
:105E800000000026B86A019008E0012300AA394604
:105E9000584600F09DFC00283ED1761C01988642B1
:105EA000F3DB97F8380040070ED520208DF800006E
:105EB000002607E0012300AA3946584600F088FC76
:105EC00050BB761CAE42F5DB00257D614246786909
:105ED0000DF101015044FCF733FC786940447861CE
:105EE00039F8020B00287FF446AF786B7969401AC5
:105EF000396A401AB969401A796A401AF969401A30
:105F0000B96AA0EB010897F83800400719D420209F
:105F10008DF80000A94612E04FF0FF3597E001240C
:105F200000AE16F8011BB868D847B8600028F3D057
:105F3000F86A401CF862641EF3D109F10109C145F9
:105F4000EDDB7B6952463946584600F041FC00289B
:105F5000E2D130208DF80000A946386A01900FE0A8
:105F6000012400AE16F8011BB868D847B8600028B5
:105F7000D2D0F86A401CF862641EF3D109F101091D
:105F800001988145ECDBBB69FA683946584600F058
:105F90001FFC0028C0D130208DF80000A946786A87
:105FA00001900FE0012400AE16F8011BB868D84735
:105FB000B8600028B0D0F86A401CF862641EF3D1C3
:105FC00009F1010901988145ECDBB869F968FB69C1
:105FD00042183946584600F0FBFB00289CD130207F
:105FE0008DF80000A946B86A01900FE0012400AEC8
:105FF00016F8011BB868D847B86000288CD0F86A3A
:10600000401CF862641EF3D109F101090198814531
:10601000ECDB97F83800400717D520208DF80000FA
:10602000A94610E0012400AE16F8011BB868D84755
:10603000B86000283FF470AFF86A401CF862641E34
:10604000F2D109F10109C145ECDB7D617D6305A851
:1060500082451CBF504600F0C7FE284615B0BDE87B
:10606000F08F2DE9FA47064682B035690A466F2A55
:1060700008BF082705D041F02000782814BF0A2760
:106080001027D6E900013C2480468946642A18BFBF
:10609000692A05D1002903DAD8F1000869EB49091A
:1060A000B9F1000F08BFB8F1000F0CD1306B50B937
:1060B000082F3BD196F83800000737D530203B2415
:1060C00085F83B0032E0CDE90089FB1740464946A0
:1060D0003A4600F0C9FEB846A8FB0023DDE9008976
:1060E000A8EB02023032A4F1010AD2B254463A2A95
:1060F00003DB9DF80830513B9A180AF805208046CA
:106100005FEA010908BFB8F1000F03D0F068611918
:106110008842D8D3082F09D196F83800000705D552
:10612000605D302802D0641E30206055C4F13C0010
:10613000B0616119F160316B884207DA081A306288
:106140004FF6EF71308F0840308710E000290ED5F0
:1061500096F8381001F01401102908D1716B72699A
:10616000891A326A891A081A0128A8BF306204B055
:10617000BDE8F0872DE9D04306460F4614464FF0A0
:106180000008DFF8389012E0E00707D542464B469A
:1061900030463946FEF7D2FF06460F4664104046A9
:1061A000494642464B46FEF7C9FF80468946002CC9
:1061B000EAD130463946BDE8D083000000002440D3
:1061C0002DE9F04F04468FB08A46D4E90001CDE9AD
:1061D000020104AF4AF0200061280BD0206B002898
:1061E00048BF062005D404BF4AF02000672801D12B
:1061F000012020636168C1F30A5040F2FF729042AF
:106200001AD1080304BF2068002808D10320A06128
:10621000AAF161001A2835D30FF2F85107E00320E4
:10622000A061AAF161001A2829D30FF2E051E068B9
:106230000322FCF785FAA4E1012816DA204600F0D3
:106240008AFE012811DB002500204AF02001612987
:106250001FD1E168302201F8012B4A1CE260BAF13B
:10626000610F0CBF782258220FE0626840F2FE31C5
:1062700061F31E52451A62604FF0FF30E5E70FF2FE
:106280008851D4E70FF28851D1E70A706169891CFF
:10629000616110B9002600256BE14AF020006128F9
:1062A00040F09580206B00284CBF2126461CDDE97C
:1062B000020136B2771CD4E900890022002300F0E5
:1062C0006BFE3ABF89F00040CDE90280CDE902893A
:1062D0002D1F8DF810200DF1110901E000F20709C2
:1062E000012F32DBDDE9020100220023FEF780FEF0
:1062F0002BD21C2102A800F067FEDDE90201FFF7A6
:1063000029F8FF1F8046012F09DBFFF70BF8024633
:106310000B46DDE9020100F081FACDE9020109F244
:106320000700072105E008F00F0200F8012D4FEAF1
:106330002818B8F1010F01DB491EF4D5491E5CBFD6
:10634000002200F8012DF9D5C8E70DF11100A9EBE5
:1063500000010DF11107B142B8BF0E4636B2300050
:106360002ED4884206DA04A9411849780829A8BF22
:106370000F2100DA002104AA821800E0761E12F82C
:106380000139401E8B42F9D00F2904D104A94118CC
:106390004A78521C4A70002802D504AF761C2D1D85
:1063A00036B2701E0CD4C119AAF13A030A78303201
:1063B000D2B23A2AA8BF9A1801F80129401EF5D591
:1063C000206B002840F1D580701E2063D1E0DDE90C
:1063D00002010022002300F0DFFD3CBF81F00041FC
:1063E000CDE902012DB247F2975068433F4990FB37
:1063F000F1F52DB2C5F10702012A04DBDDE9020146
:10640000FFF7B8FE25E0C2F1000B0026384FDFF899
:10641000E490984614E05FEACB7007D542464B46BD
:1064200030463946FEF78AFE06460F464FEA6B0BAA
:106430004046494642464B46FEF780FE8046894626
:10644000BBF1000FE7D1DDE9020132463B46FEF722
:10645000ABFCCDE902014AF0200066280CBF05F133
:106460000A000620216B4618142EA8BF13263020E0
:106470008DF810000DF11107DFF87C90012E3DDB47
:10648000DDE90201FEF77CFF07F1080104220A237F
:10649000B0FBF3F303EB8307A0EB4700303001F8C8
:1064A000010D0A20B3FBF0F000EB8007A3EB4703DC
:1064B000303301F8013D521EE9D1083E01F10807D1
:1064C000012EDBDBDDE90201FEF75AFFFEF734FFA8
:1064D00002460B46DDE9020100F0A0F900224B461E
:1064E000FEF72CFECDE90201CAE700BFA08601003D
:1064F0000000F03F0000244084D797410DF11100C7
:10650000381A0DF1110702E0401E6D1E7F1C39780C
:106510003029F9D04AF02001662902D12DB2691C38
:1065200003E065290CBF01210021226B8E1836B2D1
:10653000B042B8BF064636B231001AD4814204DAFE
:10654000C85D3528A8BF392000DA3020CA19521E8C
:1065500000E0761E12F80139491E8342F9D039282D
:1065600002D1C85D401CC855002902D57F1E761C8B
:106570006D1C2DB2009533B23A465146204600F0CC
:1065800003F80FB0BDE8F08F2DE9F04786B006465E
:106590008A4690461D4600F0BAFD406A376B90F877
:1065A0000090012D02DA01250FF26C284AF020003C
:1065B000BDF93840662808BF641C12D0672875D121
:1065C00014F1040F78DBBC4276DA96F83800641CCC
:1065D000000702D4BD42B8BF2F4624B23F1B48BFBC
:1065E0000027F068B16924B2012C21DA30234A1C5B
:1065F0000B54012F03DA96F83810090702D502F878
:106600000090521CB261E742B8BF7C4224B26142A2
:10661000E7197162AF42B8BF3D462DB2F5612A4617
:10662000B36941461818FCF78BF8781BB062B8E0E4
:106630000818A54216DA2A464146FCF781F8B169E6
:106640006918B161601B7062012F03DA96F8380097
:10665000000705D5F06801F80090F069401CF06172
:10666000B7629EE022464146FCF76AF8B0692018FE
:106670002D1B012F03DA96F83810090703D5F168AE
:1066800000F80190401C2DB2B061AF42B8BF3D464A
:10669000F3682DB22A4604EB0801C018FCF750F845
:1066A000B0692818B061781B70627AE050466128A2
:1066B00014D14FF0700A15E0BD4204DA96F8381094
:1066C000090758BF2F467F1E48BF0027BAF1670F42
:1066D00014BF4FF0450A4FF0650A03E0412808BF98
:1066E0004FF0500AB169F06818F8013B0B544A1C8E
:1066F000012F05DA96F83810090758BFB26115D591
:1067000002F80090531CB361012F0FDB6D1E2DB2F8
:10671000AF42B8BF3D462DB22A4641461818FCF795
:106720000FF8B0692818B061781B7062B069F16821
:1067300000EB0108200008F801AB03D42B2008F877
:10674000010B03E02D2108F8011B4442002502AF94
:1067500008E00A2200A800F0F3FC019807F8010BFA
:106760006D1C009C21B20129F3DA022D06DA4AF0F1
:106770002000652804BF302008F8010B4DB93020F7
:1067800008F8010B07E06D1E02A8285C303008F8FD
:10679000010B012DF7DAB069F1684018A8EB000091
:1067A000F06196F8380000F0140010280DD17069DF
:1067B000B1690818716A0818F1690818B16A0818EF
:1067C000716B8842BCBF081A306206B0BDE8F08722
:1067D000F8B504460D4616461F46002004E0E86A58
:1067E000401CE8627F1E002047B116F8011BA86814
:1067F000A047A8600028F2D14FF0FF30F2BD0000A2
:1068000000000000000000006E616E004E414E006E
:10681000696E6600494E46003000000070B44FF0CB
:10682000004591EA030F44BF6B40FEF70BBA00BF6F
:10683000841A71EB030604D26E40001BB141121999
:1068400073414FF4001C1CEB410F34BF7CEB43063B
:1068500084E00C0DA4EB1356362E7DDC012E43DCB8
:1068600045EAC32343EA525312BFD20292025B08A5
:10687000240545EAC12141EA5051D2EBC02099419B
:1068800025D407D1B0FA80F610FA06F164D00020C2
:10689000203608E0B1FA81F6B140C6F1200220FAB4
:1068A00002F21143B0404FEAF474B4EB465434F0B2
:1068B00001064FEA74040AD8D6F50016760D04F0E6
:1068C0000044F04061FA06F25040F1404840C00AEE
:1068D00040EA415021F0004128BF5FEA500550F1E5
:1068E000000044EBD12137E045EAC323DB0A45EA47
:1068F000C121C90AB6F120050EDD42EA0242120C9E
:10690000C5F1200603FA06F6EB4042EA06056D42A1
:10691000984161F100010DE062FA06F5F240554040
:1069200063FA06FC82EA0C02F3405A406D42904141
:1069300061EB030111F4801F05D1641E620502D0D2
:106940006D004041494121F48011430875F1004335
:1069500050F1000041EB045170BC70471CEB410F3B
:1069600015D223F0004352EA43060BD04FEA4C0CF9
:10697000BCEB410F04D80C0D661E342EB7DDEBE7DF
:10698000801A994150EA410608BF0021E4E708BF98
:106990001CEB430F28BF6FF00001DDE72DE9F04F3E
:1069A00085B080460D4614461E001CBF0020306096
:1069B000474600E07F1C387800F0D3FB0028F9D16F
:1069C00038782D2816BF2B2817F8019B4FF02B097C
:1069D000002C44D4012C42D0252C40DA012C0ADBB7
:1069E000102C04BF3878302802BF787840F020009F
:1069F00078280ED10AE03878302818BF0A2408D148
:106A0000787840F02000782802D11024BF1C00E0E4
:106A10000824039700E07F1C38783028FBD00297C9
:106A20000FF294004FF0000A8DF8040009E09DF881
:106A30000410CDF800A0401A5FFA80FB04FB0ABAEC
:106A40007F1C387800F097FB014622460FF2680061
:106A500000F032F90028EAD10398B84204D10DB110
:106A6000C5F80080002022E00FF274010298615CFA
:106A7000381A401A13D4012807DABAEB0B0004D3F2
:106A80000099B0FBF4F0884209D000F07FFB22218E
:106A900001600EB1012030604FF0FF3A04E0B9F11F
:106AA0002D0F08BFCAF1000A05B12F60504605B08E
:106AB000BDE8F08F002371E730313233343536379B
:106AC00038396162636465666768696A6B6C6D6EAC
:106AD0006F707172737475767778797A0000000040
:106AE00000002115110E0D0C0B0B0A0A09090909EA
:106AF000090808080808080807070707070707071D
:106B000007070707070000002DE9F14D87B006468B
:106B1000884617461D4607A800F03EFB04460DB107
:106B20000021296020F00800012833D102200090C4
:106B300004AB07994246304600F0C8FB060003D17B
:106B40000020CDE902001DE00598FEF7EBFBCDE942
:106B50000201022E16DB0DF11808761EDDE9022374
:106B600000203549FEF7EAFA824658F8040B8B46B6
:106B7000FEF7D8FB52465B46FEF75AF8CDE9020114
:106B8000761EEBD10498C219DDE902012B4600F014
:106B90008BFC42E0022835D1009004AB07994246B5
:106BA000304600F065FD060003D10020CDE902006B
:106BB0001DE00598FEF7B6FBCDE90201022E16DBBB
:106BC0000DF11808761EDDE9022300201B49FEF7AF
:106BD000B5FA824658F8040B8B46FEF7A3FB5246E3
:106BE0005B46FEF725F8CDE90201761EEBD104994C
:106BF00002A800F0E9F9DDE902012B463A4600F06F
:106C000053FC0AE0032802D100200D4905E00428C6
:106C100006D14FF0FF306FF00041CDE9020102E0F4
:106C20000020CDE902002007DDE9020148BF81F024
:106C3000004108B0BDE8F08D65CDCD410000B04108
:106C40000000F07F00235FE7F8B504460D461646C6
:106C50001F4600F01AFE3B4632462946204601B048
:106C6000BDE8F04000F027BE0278C9B28A421AB1EE
:106C70001CBF10F8012FF9E718BF00207047000073
:106C800000F10103810704D010F8011B89B18107CD
:106C9000FAD10268B2F10131914311F0803F04BF93
:106CA00050F8042FF6E710F8011B11B110F8011B82
:106CB000FBE7C01A70470000C9B2830706D0521E16
:106CC00022D310F8013B9942F7D11FE0083A13D3C1
:106CD00002F1040241EA012141EA014150F8043B7A
:106CE000121F21BF4B40A3F1013C2CEA030C1CF006
:106CF000803FF3D0C9B2001F083210F8013B521E8A
:106D000028BF91EA030FF8D818BF0120401E704732
:106D100080B500F0BAFD012002BD000070B5054647
:106D200005F10F00C408E400C046C046A54232D2B7
:106D3000082C04D2082402E0083000F055F822485C
:106D4000026811000CD1011D0A6802B31368A34246
:106D500038BF111DF8D310E01D68A5420DD2191DD2
:106D60000B68002BF8D11268011D00E0191D0B689B
:106D700093420CD01D68A542F8D361B10D682A6812
:106D8000A2F10803A3420AD26A680A600FE000F089
:106D9000B5FD0028D0D1C046C046002070BD6319A3
:106DA0000B60121B6E685E600B681A602C600968CD
:106DB00000291DBF4A68002A091D00210160C04644
:106DC000C04605F1080070BDA804002070B5044657
:106DD0000D46164600F059FD324629462046BDE8CC
:106DE000704000F05BBD000000B9704710B5A0F125
:106DF00008042068082833D310F0070F30D1C046AC
:106E0000C0461848416809B18C4203D261604460B1
:106E100017E019464B680BB1A342FAD30A6853181E
:106E20009C421BD3A34204D123689A180A600C46E3
:106E300007E04A681AB123681B199A420ED36260B0
:106E40004C60616851B1226813198B4206D100234E
:106E5000036008688018206048686060C046C046CB
:106E600010BD0000A80400201B4213D1094236D1F6
:106E70002AB18446B0FBF2F002FB10C2704700F06A
:106E800053BDFCD30022002370470B0002000021F9
:106E900000207047904271EB030CF6D370B5B1FA45
:106EA00081F4B3FA83F52C1BA340C4F1200532FA18
:106EB00005F63343A2405FF00046E64002E05B087F
:106EC0005FEA3202841A71EB030524BF204629468B
:106ED0007641F4D302000B003000002170BD012A7E
:106EE000CFD970B5140C20D0B1FA81F4B2FA82F582
:106EF000C4F120046419B4F12006D6D3B2405FF087
:106F00000044F440002502E052085FEA3303C61A49
:106F100071EB020E24BF3046714664416D41F3D3DC
:106F200002000B002000290070BD0C46B1FBF2F1FD
:106F300002FB11452D0445EA1045B5FBF2F402FBB6
:106F4000145580B240EA0545B5FBF2F002FB105241
:106F500040EA044070BD30B4436803F000420121B0
:106F60001B031B0B436004BF0368002B08D10DE01B
:106F70000368DD0F45EA440444605B000360491E7A
:106F80004468E302F4D523031B0B436043681A43B0
:106F90004260084630BC70474FF4001C1CEB410FA8
:106FA00094BF1CEB430F09E041EA030C50EA4C0C80
:106FB00052EA0C0C03D2994208BF9042704714BFAA
:106FC0008B4282427047000070B504460D466068EF
:106FD000C0F30A5040F2FF71884207D16068000395
:106FE00004BF2068002817D0022070BD20B92046B9
:106FF000FFF7B1FF012867DA012D0FDB40F2FF71C7
:10700000091A8D420AD36068002847BF00202F4923
:1070100000202F49C4E90001012070BD4142A9426E
:10702000616806DA6FF31E51401941EA0050606052
:1070300041E0401E63680122451962F31F5305F1C8
:10704000350001F000416360352803D36160002002
:10705000206070BD002215F11F0F04DA2268236042
:10706000002020356060684213D0521E256892418E
:10707000C0F12003D2439D4045EAD272256866687C
:10708000C54006FA03F32B432360636823FA00F03C
:107090006060606808436060B2F1004F03D80DD1B2
:1070A0002078C0070AD52068401C2060206828B9D5
:1070B0006068401C60604FF0FF3070BD60688842BF
:1070C00004BF20680028F6D1002070BD0000F0FF4A
:1070D0000000F07F80B5134800F027FC0FF2480154
:1070E000016041608160C1600161416181610FF2B5
:1070F0003C0242628162C162016341630FF230026D
:1071000082630FF23402C2630164416401BD10B5B1
:10711000044800F00AFC0446206808B9FFF7DAFFCB
:10712000204610BD00000020000000002E000000DE
:1071300066616C7365000000747275650000000084
:1071400091FBF2F303FB1211C0E90031704710B557
:107150000446012000F090FB2046BDE8104000F0FE
:10716000E5BB10B50446012000F086FB2046BDE8D3
:10717000104000F0E6BB10B50446012000F07CFB97
:107180002046BDE8104000F0E6BB0000014800F0DA
:10719000CCBB00001C0100202DE9F84304460D463D
:1071A0002668002700E0761C3078FFF7DAFF002819
:1071B000F9D130782D280CBF08272B2800D1761C58
:1071C000307840F020016E2929D1761C16F8010B89
:1071D00040F02000612802BF16F8010B40F02000AB
:1071E0006E2802D0266800274CE0B046042798F8A5
:1071F0000000282846D118F8019F4846FFF7A7FF4E
:107200000028F8D1A9F130000A28F4D398F800003A
:107210005F28F0D0292835D108F1010632E069292C
:1072200033D1761C16F8010B40F020006E2802BF07
:1072300016F8010B40F02000662802D026680027CF
:1072400020E0304647F00307017841F0200169292A
:1072500002BF10F8011F41F020016E2912D110F871
:10726000011F41F02001692902BF10F8011F41F000
:107270002001742906D110F8011F41F0200179295D
:1072800008BF461CF5B12E601CE0302802BF7078A4
:1072900040F02000782813D1B01C01782E2908BFB7
:1072A000401C0078A0F16101062921BFA0F1410135
:1072B000062930380A2803D2B61C47F0020701E03D
:1072C00047F0010726603846BDE8F2832DE9F04F0C
:1072D0008DB08146169800EBC0080D4692461E46BA
:1072E0004FF0000BB8F12E0FA8BF4FF02D08C6F8D5
:1072F00000B0C6F804B0002701E06D1C0127287813
:107300003028FAD0002401A804E03168491C31601B
:107310006D1C01272978A1F130020A2A0AD30091B5
:10732000FFF7F5FE406A01780098884208BF6D1C9F
:1073300074B90AE0A045E8DB30392154641CE7E762
:107340003068401E30606D1C012728783028F7D047
:107350002878A0F130010A2912D3A04525DA01A826
:1073600018F80000052806DB01A8404410F8011CAD
:10737000491C00F8011C44463068401C306014E091
:10738000A04506DB01A930386054641C3068401EFB
:1073900030606D1C0127DBE701A8201810F8010CF4
:1073A00048B93068401C3060641E012CF4DA14B90E
:1073B0008DF804B00124002F58D0092294FBF2F27A
:1073C000C4F1090002EBC2021218092092FBF0F08E
:1073D000002100EBC000101A0DD04FF0010B0AE0A5
:1073E00056F82B30085C03EB830300EB430046F8B0
:1073F0002B00521C491CA1420BDA092392FBF3F328
:1074000003EBC30301A8D31AEAD1085C0BF1010B0B
:10741000EDE7287840F02000652827D1284615F8A8
:10742000011F2B2916BF2D2915F8011B2B214FF009
:10743000000C0023134A09E0934204DA03EB8304AF
:107440000EEB4403303B6D1C4FF0010C95F800E04F
:10745000AEF130040A2CEFD32D2908BF5B4231680E
:1074600059183160BCF1000F08BF0546BAF1000F92
:1074700003D007B1A946CAF8009058460DB0BDE840
:10748000F08F00BF00E1F50530303A3030303A304F
:10749000303A30303A30303A30303A30303A3030BA
:1074A00030000000000000002DE9FB4582B016000E
:1074B0009A4600F0A880DDE902230020002100F0B8
:1074C00051FA00F0A0800024514D002E45D576429F
:1074D0000FF254174FF008080DE0F00707D5D7E971
:1074E000002320462946FDF729FE04460D4676086E
:1074F0000837A8F10108002E18BFB8F1000FECD131
:1075000002A900A800F03EFADDE9020122462B465E
:10751000FDF74AFCCDE90201BDF9001002A8FFF712
:1075200053FD07005ED5002E5ED0002E5AD002A972
:1075300000A800F027FADDE90201364A364BFDF7D4
:10754000FDFDCDE90201BDF9001002A8FFF73CFDE9
:10755000070048BF761EE8D444E0012E42DB0FF25C
:10756000C8074FF00808F00707D5D7E900232046E1
:107570002946FDF7E3FD04460D4676100837A8F1CD
:107580000108012E02DBB8F1000FECD102A900A81E
:1075900000F0F8F9DDE9020122462B46FDF7CEFDA9
:1075A000CDE90201BDF9001002A8FFF70DFD0700AB
:1075B00018D5012E18DB00E0761E012E12DB02A981
:1075C00000A800F0DFF9DDE90201144A144BFDF7D1
:1075D000B5FDCDE90201BDF9001002A8FFF7F4FCEA
:1075E0000700E9D43FB20FB1012F0CD1FFF7CEFD58
:1075F00022210160BAF1000F05D0DAF8000040F056
:107600000100CAF80000DDE9020105B0BDE8F0851F
:107610000000F03F436FAC642806C80A3CBF737F8C
:10762000DD4F157500000000000000000000244040
:107630000000000000005940000000000088C34026
:107640000000000084D797410080E03779C34143B0
:10765000176E05B5B5B89346F5F93FE9034F384DB8
:10766000321D30F94877825A3CBF737FDD4F157564
:107670002DE9F14F8AB00E461498C0EBC00B90462E
:107680001D464FF0000ABBF1240FA8BF4FF0230B9B
:10769000C5F800A0C5F804A0002701E0761C01276A
:1076A00030783028FAD00FF2A010002400900DF1AD
:1076B000040904E02868401C2860761C0127317802
:1076C00016220FF28410FFF7F7FA50B1A345F1DB51
:1076D0000099401A0FF28811405C04F80900641CFC
:1076E000EBE796F80090FFF712FD406A00788145BD
:1076F00008BF761C44B904E02868401E2860761C48
:10770000012730783028F7D0317816220FF2381060
:10771000FFF7D2FA80B1A3450BDB0FF22C11401A10
:107720000FF23C11405C01A96054641C2868401EA3
:107730002860761C0127E7E7A34519DA01A81BF8A2
:107740000000082806DB01A8584410F8011C491C59
:1077500000F8011C5C462868401C286008E001A86D
:10776000201810F8010C48B92868401C2860641ED5
:10777000012CF4DA14B98DF804A0012428688000E3
:107780002860002F53D0072294FBF2F2C4F10701C6
:10779000C2EBC2025118072291FBF2F20020C2EBA9
:1077A000C2028A1A06D04FF0010A03E045F82A20E7
:1077B000491C401CA0420FDA01ABC25C072391FBBD
:1077C000F3F3C3EBC303CB1A0EBF0AF1010A55F85A
:1077D0002A3002EB0312E9E7307840F020007028ED
:1077E00025D1304616F8011F2B2916BF2D2916F872
:1077F000011B2B2100220023124C09E0A34205DAD1
:1078000003EB83020CEB4202A2F13003761C01224F
:1078100096F800C0ACF1300EBEF10A0FEED32D2960
:1078200008BF5B4229685918296002B90646B8F1B9
:10783000000F03D007B90A9EC8F8006050460BB08D
:10784000BDE8F08F00E1F50530313233343536379D
:1078500038396162636465664142434445460000CD
:10786000000102030405060708090A0B0C0D0E0FA0
:107870000A0B0C0D0E0F000010B50446DFF81800BF
:1078800000F053F850F8240010BD80B5DFF8080070
:1078900000F04BF8806902BD9000002030B430B990
:1078A0000FF24800D0E90045C2E900451BE0017035
:1078B000012030BC704730B431B90FF23800D0E944
:1078C0000045C3E900450EE01AB930BC6FF0010075
:1078D000704708B10A7802800978481E804130BCA0
:1078E000C043C00F7047002030BC7047000000004C
:1078F00000000000000000000000000007490868C8
:1079000008B1002070470648C008C000086005495B
:10791000C908C900091A0160704700BFBC040020F3
:10792000EF0C0020E814002070477047A0F16101BF
:107930001A2904D341381A288041C00F704701200A
:107940007047A0F10901052901D3202801D10120A8
:10795000704700207047A0F141011A2938BF20303C
:107960007047000090420CD141EA030C50EA4C0CE5
:1079700007D0994205D14FF4001C1CEB410F38BFD2
:107980008942704738B50C4605466068C0F30A5016
:1079900040F2FF7188420BD100202880606800030C
:1079A00004BF2068002801D0022032BD012032BD72
:1079B000012804DA2046FFF7CEFA01280ADA6268C5
:1079C00040F2FE3161F31E526260401A28804FF08F
:1079D000FF3032BD0020288032BD000000000000D2
:1079E0000000000000000000000000000000000097
:1079F0000000000000000000000000000000000087
:107A00000000000000000000000000000000000076
:107A1000E003E003E003E003E003E003E003E0034E
:107A2000C003C003C001C001C001C001C00100000B
:107A300000000000E003E003E0030000000000009D
:107A4000000000003C1E3C1E3C1E3C1E3C1E3C1E1A
:107A50003C1E0000000000000000000000000000CC
:107A60000000000000000000000000000000000016
:107A70000000000000000000CE01CE03DE039E03E4
:107A80009C039C07FF3FFF7F3807380F780F780F64
:107A9000780EFFFFFFFFF01EF01CE01CE03CE03D15
:107AA000E03900000000000000000000FC03FE0FB1
:107AB000EE1FE01EE01EE01EE01EE01FE00FE007EC
:107AC000F003FC01FE01FE01FE01FE01FE01FE01CC
:107AD000FE3DFC3FF00FE001E0010000000000006F
:107AE000033E07F78FE78EE79EE3BCE3B8E7F8E7CE
:107AF000F0F7E03FC001FF03FF07F307F30FF31EAA
:107B0000F33CF338F3787FF03FE000000000000022
:107B100000000000E007F80F780F781F781F781F2B
:107B2000780FF00FE00F801FC37FC3FBE7F3F7F17F
:107B3000F7F0FFF07FF03EF87F7CFF3FEF1F000083
:107B40000000000000000000E003E003E003E003A9
:107B5000E003C003C00100000000000000000000BE
:107B60000000000000000000000000000000000015
:107B70000000000000000000000000003F007C004A
:107B8000F001E001C003C00780078007800F000FED
:107B9000000F000F000F000F000F800F80078007FD
:107BA000C007C003E001F0017C003F000F000000AF
:107BB000007E001FC007C003E001F001F000F000EC
:107BC000F800780078007800780078007800F800F5
:107BD000F000F000F001E001C003C007001F007ECC
:107BE00000780000E003C003C001CE39FF3F7F3FB3
:107BF00020037003F807780F3C1F380600000000D0
:107C00000000000000000000000000000000000074
:107C10000000000000000000000000000000000064
:107C200000000000C001C001C001C001C001C001CE
:107C3000C001FFFFFFFFC001C001C001C001C001C2
:107C4000C001000000000000000000000000000073
:107C50000000000000000000000000000000000024
:107C60000000000000000000000000000000E00331
:107C7000E003E003E003E001E001E001C001800374
:107C800000000000000000000000000000000000F4
:107C9000000000000000FE3FFE3F0000000000006A
:107CA00000000000000000000000000000000000D4
:107CB00000000000000000000000000000000000C4
:107CC00000000000000000000000000000000000B4
:107CD000000000000000E003E003E003E003000018
:107CE00000000000000000000F000F001E001E003A
:107CF0003C003C0078007800F000F000E001E0017A
:107D0000C003C00380078007000F000F001E001E85
:107D1000003C003C0078007800F00000F007F80F0D
:107D20007C1F3E3E1E3C1F7C1F7C0F780F780F7817
:107D30000F780F780F780F781F7C1F7C1E3C3E3E1B
:107D40007C1FF80FF007000000000000000000009A
:107D5000F000F007F03FF03FF001F001F001F0011A
:107D6000F001F001F001F001F001F001F001F0018B
:107D7000F001F001F001FF3FFF3F000000000000B4
:107D800000000000E00FF83F7C3C3C003E003E005D
:107D90003E003C003C007C00F800F001E003C0071E
:107DA0008007000F001E003E003CFE3FFE3F00002B
:107DB0000000000000000000F00FF81F7C1C3E00D7
:107DC0003E003E003C003C00F800F00FF80F7C0045
:107DD0003E001E001E001E001E003E007C1CF81F00
:107DE000E01F000000000000000000007800F80024
:107DF000F800F801F803F807F807780F781E781EE6
:107E0000783C78787878FFFFFFFF7800780078007A
:107E100078007800780000000000000000000000FA
:107E2000FC1FFC1FFC1F001E001E001E001E001E6B
:107E3000E01FF81FFC007C003E003E001E003E00DC
:107E40003E003C007C1CF81FE01F0000000000000A
:107E500000000000FC01FE078E0F001F001E003E08
:107E6000003C003CF83DFC3F3E7F1F7E0F3C0F3C3A
:107E70000F3C0F3C0F3E1F1E3E1FFC0FF003000087
:107E80000000000000000000FF3FFF3FFF3F0F0029
:107E90001E001E003C0038007800F000F000E001F9
:107EA000E001C003C0038007800F800F000F001F98
:107EB000001F00000000000000000000F807FC0F99
:107EC0003E1F1E1E1E3E1E3E1E1E3C1FF80FF007CC
:107ED000F80FFC1E3E3E1F3C1F7C0F7C0F7C1F3C9E
:107EE0003E3FFC1FF0070000000000000000000003
:107EF000F007F80F7C1E3E3C1E3C1F7C1F7C1F7C45
:107F00001F7C1F3C3F3EFF1FEF071F001E001E008F
:107F10003E003C00F838F03FE01F00000000000089
:107F20000000000000000000000000000000000051
:107F3000E003E003E003E0030000000000000000B5
:107F4000000000000000E003E003E003E0030000A5
:107F50000000000000000000000000000000000021
:107F600000000000E003E003E003E0030000000085
:107F700000000000000000000000E003E003E00358
:107F8000E003E001E001E001C00380030000000025
:107F9000000000000000000003000F003F00FC0094
:107FA000F003C00F003F00FE003FC00FF003FC00D5
:107FB0003F000F0003000000000000000000000070
:107FC00000000000000000000000000000000000B1
:107FD00000000000FFFFFFFF000000000000FFFFA7
:107FE000FFFF000000000000000000000000000093
:107FF0000000000000000000000000000000000081
:1080000000E000F8007E801FE007F8017E001F00FE
:108010007E00F801E007801F007E00F800E000000D
:108020000000000000000000F01FFC3F3E381F3839
:108030001F381E001E003C007800F000E001C00365
:10804000C003C007C007000000000000C007C00751
:10805000C00700000000000000000000F803FE0F51
:108060001E1F0F3E7F3CFF78EF79C773C7F38FF376
:108070008FF38FF39FF39FF3FF73FF7BF779003C40
:108080001C1FFC0FF80300000000000000000000AF
:10809000000000000000E003E003F007F007F00735
:1080A000780F780F7C0E3C1E3C1E3E3CFE3FFF3F8F
:1080B0001F780F780FF007F007F0000000000000B5
:1080C00000000000000000000000F83FFC3F3E3CC4
:1080D0001E3C1E3C1E3C3E3C7C3CF03FF83F7E3C40
:1080E0001F3C1F3C0F3C0F3C1F3CFE3FF83F000075
:1080F0000000000000000000000000000000FF0180
:10810000FF07871F003E003C007C00780078007865
:1081100000780078007C007C003E003F831FFF0752
:10812000FF0100000000000000000000000000004F
:108130000000F07FFC7F7E781F781F780F780F7823
:108140000F780F780F780F780F780F781F781E78D8
:108150007E78F87FE07F0000000000000000000053
:10816000000000000000FF3FFF3F003E003E003ED9
:10817000003E003E003EFE3FFE3F003E003E003E11
:10818000003E003E003EFF3FFF3F000000000000B9
:1081900000000000000000000000FF1FFF1F001E85
:1081A000001E001E001E001E001EFF1FFF1F001EDF
:1081B000001E001E001E001E001E001E001E0000ED
:1081C0000000000000000000000000000000FE03AE
:1081D000FF0F871F003E007C007C007800F800F84D
:1081E0007FF87FF80F780F7C0F7C0F3E8F1FFF0FFB
:1081F000FE0300000000000000000000000000007E
:1082000000001F7C1F7C1F7C1F7C1F7C1F7C1F7C31
:108210001F7CFF7FFF7F1F7C1F7C1F7C1F7C1F7CC0
:108220001F7C1F7C1F7C000000000000000000007D
:10823000000000000000FF3FFF3FE003E003E00319
:10824000E003E003E003E003E003E003E003E00316
:10825000E003E003E003FF3FFF3F000000000000F9
:1082600000000000000000000000FC1FFC1F7C005C
:108270007C007C007C007C007C007C007C007C001E
:108280007C007C0078007800F838F03FC03F0000A8
:1082900000000000000000000000000000001F3C83
:1082A0001E3C3C3C783CF03CE03DE03FC03F803F22
:1082B000C03FE03FF03DF03C783C7C3C3E3C1F3C06
:1082C0000F3C000000000000000000000000000063
:1082D0000000003E003E003E003E003E003E003EEC
:1082E000003E003E003E003E003E003E003E003E9E
:1082F000003EFF3FFF3F00000000000000000000C4
:108300000000000000001FF81FFC1FFC3FFE3FFEA6
:108310003FFE7FFF77FF77FFF7F7E7F7E7F3E7F336
:10832000C7F307F007F007F007F0000000000000B7
:10833000000000000000000000000F7C0F7C0F7E9A
:108340000F7F0F7F8F7F8F7FCF7FEF7BEF79FF795D
:10835000FF78FF787F783F783F781F781F7800009C
:108360000000000000000000000000000000F00716
:10837000FC1F3E3E1F7C0F780F780FF80FF80FF8A8
:108380000FF80FF80FF80F780F781F7C3E3EFC1F98
:10839000F0070000000000000000000000000000E6
:1083A0000000FC3FFF3F1F3E0F3E0F3E0F3E0F3EC3
:1083B0001F3E3F3EFC3FF03F003E003E003E003E81
:1083C000003E003E003E00000000000000000000F3
:1083D000000000000000F007FC1F3E3E1F7C0F78ED
:1083E0000F780FF80FF80FF80FF80FF80FF80F7855
:1083F0000F781F7C3E3EFC1FF8077C003F000F00FB
:1084000003000000000000000000F03FFC3F7E3C45
:108410003E3C1E3C1E3C3E3C3C3CFC3CF03FE03FB6
:10842000F03DF83C7C3C3E3C1E3C1F3C0F3C0000B9
:108430000000000000000000000000000000FC0739
:10844000FE1F0E3E003C003C003C003EC01FF80FEB
:10845000FE037F001F000F000F001F203E3CFC3F6B
:10846000F01F0000000000000000000000000000FD
:108470000000FFFFFFFFE003E003E003E003E00391
:10848000E003E003E003E003E003E003E003E003D4
:10849000E003E003E0030000000000000000000033
:1084A0000000000000000F7C0F7C0F7C0F7C0F7C15
:1084B0000F7C0F7C0F7C0F7C0F7C0F7C0F7C0F7C64
:1084C0001E3C1E3C3E3EFC1FF0070000000000006A
:1084D0000000000000000000000007F007F007F8AF
:1084E0000F780F7C1E3C1E3C1E3E3C1E3C1F781F1E
:1084F000780FF80FF007F007F007E003E003000043
:10850000000000000000000000000000000003E088
:1085100003F003F007F0E7F3E7F3E7F3E773F77B24
:10852000F77FFF7F7F7F7F7F7E7F7E3F3E3E3E3EA9
:108530003E3E0000000000000000000000000000BF
:10854000000007F80F7C1E3E3E3E3C1FF80FF00770
:10855000E007E003E003F007F80F7C0F7C1E3E3CD1
:108560001F780F780FF000000000000000000000EE
:1085700000000000000007F807780F7C1E3C1E3E3C
:108580003C1F780FF80FF007E003E003E003E0037F
:10859000E003E003E003E003E0030000000000006C
:1085A00000000000000000000000FF7FFF7F0F00C0
:1085B0001F003E007C00F800F000E001E003C0076F
:1085C000800F000F001E003E007CFF7FFF7F000039
:1085D0000000000000000000FF0780078007800700
:1085E0008007800780078007800780078007800753
:1085F0008007800780078007800780078007800743
:10860000800780078007FF07FF07000000780078D9
:10861000003C003C001E001E000F000F800780077A
:10862000C003C003E001E001F000F0007800780032
:108630003C003C001E001E000F000F000700000061
:10864000F07FF000F000F000F000F000F000F0002B
:10865000F000F000F000F000F000F000F000F0009A
:10866000F000F000F000F000F000F000F000F07F0B
:10867000F07F0000C000C001C001E003E003F0078C
:10868000F0077807780F380F3C1E3C1E1E3C1E3C3E
:108690000F380F780778000000000000000000008D
:1086A00000000000000000000000000000000000CA
:1086B00000000000000000000000000000000000BA
:1086C00000000000000000000000000000000000AA
:1086D0000000FFFFFFFF000000000000F0000000AE
:1086E000000000000000000000000000000000008A
:1086F000000000000000000000000000000000007A
:108700000000000000000000000000000000000069
:10871000000000000000000000000000F80FFC3F17
:108720007C3C3E003E003E00FE07FE1F3E3E3E7C7F
:108730003E783E7C7E7CFF3FCF1F000000000000A3
:1087400000000000003C003C003C003C003C003CC1
:10875000F83DFE3F3E3F1F3E0F3C0F3C0F3C0F3CA1
:108760000F3C0F3C1F3C1E3C3E3FFC3FF03B0000DB
:1087700000000000000000000000000000000000F9
:1087800000000000FE03FF0F871F003E003E003C7C
:10879000007C007C007C003C003E003E871FFF0FF9
:1087A000FE03000000000000000000001F001F008A
:1087B0001F001F001F001F00FF07FF1F3F3E1F3C41
:1087C0001F7C1F7C1F7C1F781F781F7C1F7C3F3CF9
:1087D0007F3EFF1FDF0F00000000000000000000D0
:1087E000000000000000000000000000F803FC0F83
:1087F0003E1F1E3E1F3C1F7CFF7FFF7F007C007CD6
:10880000003C003E071FFF0FFE03000000000000B9
:1088100000000000FF01E103C003C007C007C0075C
:10882000FF7FFF7FC007C007C007C007C007C007A2
:10883000C007C007C007C007C007C007C0070000C7
:108840000000000000000000000000000000000028
:1088500000000000EF07FF1F7F3E1F3C1F7C1F7CB6
:108860001F781F781F781F7C1F7C3F3C7F3EFF1FB7
:10887000DF0F1E001E001E007C38F83F003C003C4D
:10888000003C003C003C003CFC3DFE3F9E3F1F3F47
:108890001F3E1F3C1F3C1F3C1F3C1F3C1F3C1F3CFE
:1088A0001F3C1F3C1F3C00000000000000000000B7
:1088B000F001F0010000000000000000E07FE07F18
:1088C000E001E001E001E001E001E001E001E001A0
:1088D000E001E001E001E001E00100000000000033
:1088E00000000000F800F800000000000000000098
:1088F000F83FF83FF800F800F800F800F800F8003A
:10890000F800F800F800F800F800F800F800F800A7
:10891000F800F000F071E07F003C003C003C003CBF
:10892000003C003C1F3C3E3C7C3CF83CF03DE03DC4
:10893000C03FC03FE03FF03DF83C7C3C3E3C1F3C2C
:108940001F3C00000000000000000000F07FF0016C
:10895000F001F001F001F001F001F001F001F0018F
:10896000F001F001F001F001F001F001F001F0017F
:10897000F001F001F0010000000000000000000024
:108980000000000000000000000000009EF7FFFF54
:10899000FFFFFFFFE7FBE7F9C7F1C7F1C7F1C7F139
:1089A000C7F1C7F1C7F1C7F1C7F10000000000002F
:1089B00000000000000000000000000000000000B7
:1089C000FC3DFE3F9E3F1F3F1F3E1F3C1F3C1F3C88
:1089D0001F3C1F3C1F3C1F3C1F3C1F3C1F3C00001A
:1089E0000000000000000000000000000000000087
:1089F00000000000F007FC1F3E3E1F3C1F7C0F786C
:108A00000F780F780F780F781F7C1F3C3E3EFC1FBD
:108A1000F00700000000000000000000000000005F
:108A20000000000000000000F83DFE3F3E3F1F3EFA
:108A30000F3C0F3C0F3C0F3C0F3C0F3C1F3C1E3EBD
:108A40003E3FFC3FF83F003C003C003C003C003C0B
:108A5000000000000000000000000000EE07FE1F04
:108A60007E3E1E3C1E7C1E781E781E781E781E7868
:108A70001E7C3E7C7E3EFE1FDE0F1E001E001E0082
:108A80001E001E00000000000000000000000000AA
:108A90007F1FFF1FE71FC71F871F001F001F001F2B
:108AA000001F001F001F001F001F001F001F0000ED
:108AB00000000000000000000000000000000000B6
:108AC00000000000FC07FE1F0E1E003E003E003F9F
:108AD000E01FFC07FE003E001E001E003E3CFC3F67
:108AE000F01F000000000000000000000000000077
:108AF0000000800780078007FF7FFF7F80078007D7
:108B0000800780078007800780078007800780072D
:108B1000C007FF03FF01000000000000000000008C
:108B20000000000000000000000000001E3C1E3C91
:108B30001E3C1E3C1E3C1E3C1E3C1E3C1E3C1E3C65
:108B40003E3C7E3CFE3EFE1FDE0F000000000000AB
:108B50000000000000000000000000000000000015
:108B600007F00F780F781E3C1E3C1E3E3C1E3C1E3C
:108B7000780F780FF00FF007F007E003E003000034
:108B800000000000000000000000000000000000E5
:108B90000000000003F0E3F1E3F3E7F3F7F3F7F38A
:108BA000F77F777F7F7F7F7F7F7F3E3E3E3E3E3EEB
:108BB0003E3E000000000000000000000000000039
:108BC00000000000000000000F7C1E3E3C3E3C1FE9
:108BD000F80FF007F007E003F007F807F80F7C1E26
:108BE0003E3E1F3C1F780000000000000000000017
:108BF00000000000000000000000000007F80F78EF
:108C00000F7C1E3C1E3C3C1E3C1E3C1F780FF80F88
:108C1000F007F007E003E003C003C003C0038007D0
:108C2000800F007F00000000000000000000000036
:108C3000FF3FFF3F1F003E007C00F800F001E00313
:108C4000C007800F001F001E003CFF7FFF7F000059
:108C50000000000000000000FE01E003C003C003AC
:108C6000C003C003E001E001E001C001C003803F98
:108C7000803FC003C001E001E001E001C003C00388
:108C8000C003C003E003FE017E000000C001C0017C
:108C9000C001C001C001C001C001C001C001C001CC
:108CA000C001C001C001C001C001C001C001C001BC
:108CB000C001C001C001C001C001C001C00100006D
:108CC000C03FE003E001E001E001E001C001C003BA
:108CD000C003C001E001FE00FE00E001C001C003CE
:108CE000C003C001E001E001E001E001E003C03F9A
:108CF000003F000000000000000000000000000035
:108D000000000000000000000000073FC77FE7737D
:108D1000FFF17EF0000000000000000000000000F5
:108D20000000000000000000000000000000000043
:108D30000000000000000000000000000000000033
:108D40000000000000000000000000000000000C17
:108D5000000C000C000C000C000C000C000C000CB3
:108D6000000C000C0000000C000C000000000000D3
:108D70000000001B001B001B001B001B000000006C
:108D800000000000000000000000000000000000E3
:108D90000000000000008019801980198019C07F30
:108DA000C07F80190033C07FC07F003300330033A1
:108DB00000330000000000000000001E003F80752E
:108DC00080650074003C001E00078005806580659A
:108DD0008075003F001E00040004000000000070C9
:108DE00000D840D8C0D880D900730006000C801B82
:108DF000C036C066C046C006800300000000000008
:108E00000000001E003F003300330033001E000C42
:108E1000C03CC066806380618063C03E801C0000EF
:108E2000000000000000000C000C000C000C000C06
:108E30000000000000000000000000000000000032
:108E40000000000000000000800000010003000698
:108E500000060004000C000C000C000C000C000CC0
:108E6000000400060006000300018000002000103E
:108E70000018000C000C00040006000600060006A6
:108E8000000600060004000C000C00180010002072
:108E90000000000C002D003F001E00330000000009
:108EA00000000000000000000000000000000000C2
:108EB00000000000000000000000000C000C000C8E
:108EC000000CC0FFC0FF000C000C000C000C0000E8
:108ED0000000000000000000000000000000000092
:108EE0000000000000000000000000000000000082
:108EF0000000000C000C000400040008000000004A
:108F00000000000000000000000000000000001E43
:108F1000001E000000000000000000000000000033
:108F20000000000000000000000000000000000041
:108F300000000000000000000000000C000C000019
:108F4000000000000000000300030003000600060C
:108F500000060006000C000C000C000C00180018A5
:108F600000180000000000000000001E003F003359
:108F7000806180618061806D806D806180618061D1
:108F80000033003F001E000000000000000000064B
:108F9000000E001E00360026000600060006000631
:108FA00000060006000600060006000000000000A3
:108FB0000000001E003F807380618061800100031B
:108FC0000006000C001800300060807F807F0000E9
:108FD000000000000000001C003E0063006300036E
:108FE000000E000E00038001800180618073003F4D
:108FF000001E00000000000000000006000E000E31
:10900000001E001E0016003600360066807F807F3E
:109010000006000600060000000000000000007FBF
:10902000007F006000600060006E007F8063800150
:10903000800180618073003F001E0000000000007E
:109040000000001E003F803380610060006E007FE2
:1090500080738061806180618033003F001E00006A
:10906000000000000000807F807F8001000300037B
:1090700000060006000C000C000C00080018001888
:1090800000180000000000000000001E003F806388
:10909000806180610021001E003F806180618061ED
:1090A0008061003F001E0000000000000000001E64
:1090B000003F00738061806180618073803F801D0C
:1090C000800180610073003F001E0000000000006E
:1090D00000000000000000000000000C000C000078
:1090E00000000000000000000000000C000C000068
:1090F0000000000000000000000000000000000070
:10910000000C000C00000000000000000000000C3B
:10911000000C000400040008000000000000000033
:1091200080008003000E003800600038000E8003CD
:1091300080000000000000000000000000000000AF
:10914000000000000000807F807F00000000807F22
:10915000807F000000000000000000000000000010
:10916000000000000000000000400070001C00072C
:1091700080010007001C007000400000000000009B
:10918000000000000000001F803FC071C060C000F0
:10919000C00180030007000E000C000C0000000C52
:1091A000000C0000000000000000001E003F8031A5
:1091B00080718063806F806D806D806F80670060DC
:1091C0000032003E001C0000000000000000000E05
:1091D000000E001B001B001B001B80318031803FF4
:1091E000803F8031C060C060C060000000000000AF
:1091F0000000007C007E0063006300630063007E6B
:10920000007E0063806180618063007F007E0000DB
:10921000000000000000001E003F803180610060FF
:109220000060006000600060006080618031003F8D
:10923000001E0000000000000000007C007F0063B2
:109240008063806180618061806180618061006392
:109250000063007E007C0000000000000000807FB2
:10926000807F0060006000600060007F007F006021
:10927000006000600060807F807F000000000000D0
:109280000000807F807F0060006000600060007FE1
:10929000007F00600060006000600060006000000F
:1092A000000000000000001E003F8031806100606F
:1092B0000060006080638063806180618031803FF6
:1092C000001E0000000000000000806180618061DD
:1092D000806180618061807F807F8061806180614A
:1092E0008061806180610000000000000000003F9C
:1092F000003F000C000C000C000C000C000C000CDB
:10930000000C000C000C003F003F000000000000BB
:1093100000008001800180018001800180018001C6
:1093200080018001806180618073003F001E000029
:10933000000000000000C0608061006300660066FD
:10934000006C0078007C00660066006380618061CC
:10935000C0600000000000000000006000600060CD
:1093600000600060006000600060006000600060FD
:109370000060807F807F0000000000000000C0715E
:10938000C071C07BC07AC06AC06AC06EC064C06071
:10939000C060C060C060C060C0600000000000002D
:1093A000000080718071807980798079806D806D16
:1093B000806D806580678067806780638063000060
:1093C000000000000000001E003F0033806180614B
:1093D0008061806180618061806180610033003FD5
:1093E000001E0000000000000000007E007F80637F
:1093F0008061806180618063007F007E006000602A
:109400000060006000600000000000000000001E1E
:10941000003F003380618061806180618061806194
:10942000806580670033803F401E00000000000020
:109430000000007E007F8063806180618063007F28
:10944000007E00660063006380618061C060000090
:10945000000000000000000E001F8031803100304D
:109460000038001E00078003806180618031003F6A
:10947000001E0000000000000000C0FFC0FF000C44
:10948000000C000C000C000C000C000C000C000C7C
:10949000000C000C000C00000000000000008061C7
:1094A00080618061806180618061806180618061B4
:1094B000806180618073003F001E0000000000009A
:1094C0000000C060C060C060803180318031001B0E
:1094D000001B001B001B000E000E000E000400000D
:1094E000000000000000C0C0C0C0C0C0C0C0C0C0FC
:1094F000C0CC804C804C805E8052805280738061F2
:1095000080610000000000000000C0C08060806139
:109510000033003B001E000C000C001E001F003B2F
:1095200080718061C0C00000000000000000C0C069
:109530008061806100330033001E001E000C000CAF
:10954000000C000C000C000C000C000000000000DF
:109550000000803F803F8001000300030006000CF4
:10956000000C0018001800300060807F807F000031
:1095700000000000000F000F000C000C000C000C9D
:10958000000C000C000C000C000C000C000C000C7B
:10959000000C000C000F000F00000018001800184D
:1095A000000C000C000C000C000600060006000673
:1095B000000300030003000000000000001E001E66
:1095C000000600060006000600060006000600066B
:1095D000000600060006000600060006001E001E2B
:1095E0000000000C000C001E0012003300338061EC
:1095F000806100000000000000000000000000008A
:10960000000000000000000000000000000000005A
:10961000000000000000000000000000000000004A
:1096200000000000E0FF0000000000380018000CFF
:10963000000000000000000000000000000000002A
:10964000000000000000000000000000000000001A
:10965000000000000000001F803F80618001801F2B
:10966000803F80618063807FC03800000000000080
:1096700000000060006000600060006E007F80738A
:1096800080618061806180618073007F006E000076
:109690000000000000000000000000000000001EAC
:1096A000003F807380610060006080618073003FD4
:1096B000001E000000000000000080018001800109
:1096C0008001801D803F8073806180618061806146
:1096D0008073803F801D000000000000000000003B
:1096E000000000000000001E003F00738061807FCA
:1096F000807F00608071003F001E000000000000BD
:109700000000C007C00F000C000C807F807F000CA1
:10971000000C000C000C000C000C000C000C0000F5
:10972000000000000000000000000000801D803FDD
:10973000807380618061806180618073803F801D63
:1097400080018063007F003E0000006000600060D8
:109750000060006F807F80718061806180618061C6
:109760008061806180610000000000000000000650
:10977000000600000000003E003E00060006000655
:1097800000060006000600060006000000000000BB
:109790000006000600000000003E003E0006000635
:1097A0000006000600060006000600060006004649
:1097B000007E003C0000006000600060006080618E
:1097C00000630066006C007C0076006300638061CB
:1097D000C0600000000000000000003E003E0006E7
:1097E0000006000600060006000600060006000649
:1097F0000006000600060000000000000000000057
:1098000000000000000080DDC0FFC0CEC0CCC0CC96
:10981000C0CCC0CCC0CCC0CCC0CC0000000000008C
:1098200000000000000000000000006F807F8071D9
:109830008061806180618061806180618061000001
:109840000000000000000000000000000000001EFA
:10985000003F807380618061806180618073003F20
:10986000001E0000000000000000000000000000DA
:10987000006E007F80738061806180618061807391
:10988000007F006E0060006000600060000000006B
:1098900000000000801D803F8073806180618061D6
:1098A00080618073803F801D800180018001800184
:1098B000000000000000000000000067803F003949
:1098C0000030003000300030003000300030000048
:1098D0000000000000000000000000000000001E6A
:1098E000803F80610060007F803F80018061007F59
:1098F000001E00000000000000000000000800182A
:109900000018007F007F00180018001800180018C9
:109910000018801F800F0000000000000000000001
:1099200000000000000080618061806180618061D2
:10993000806180618063807F803D000000000000C6
:1099400000000000000000000000C0608031803195
:109950008031001B001B001B000E000E00060000E3
:10996000000000000000000000000000000080DD9A
:1099700080DD80DD0055005500550077007700221E
:1099800000220000000000000000000000000000B5
:109990000000806100330033001E000C000C001E2C
:1099A0000033003380610000000000000000000070
:1099B0000000000080618061803100330033001BB3
:1099C000001B001B000E000E000E001C007C00702F
:1099D00000000000000000000000C07FC07F800188
:1099E00000030006000C00180030C07FC07F00009C
:1099F0000000000080038007000600060006000645
:109A00000006000E001C001C000E000600060006EA
:109A10000006000680078003000600060006000618
:109A20000006000600060006000600060006000606
:109A30000006000600060006000600060038003C8E
:109A4000000C000C000C000C000C000E00070007BE
:109A5000000E000C000C000C000C000C003C003848
:109A6000000000000000000000000000000080383E
:109A7000807F0047000000000000000000000000A0
:109A800000000000000000000000000000000000D6
:109A90000000000000000000001000100010001086
:109AA0000010001000000010000000000028002836
:109AB000002800000000000000000000000000007E
:109AC00000240024007C00240048007C004800485A
:109AD000000000000038005400500038001400540A
:109AE00000540038001000000020005400580030DE
:109AF0000028005400140008000000000010002896
:109B00000028001000340048004800340000000025
:109B10000010001000100000000000000000000015
:109B2000000000000008001000200020002000209D
:109B3000002000200010000800200010000800088D
:109B4000000800080008000800100020001000387D
:109B500000100028000000000000000000000000CD
:109B60000000000000100010007C00100010000039
:109B700000000000000000000000000000000000E5
:109B800000000010001000100000000000000000A5
:109B9000000000380000000000000000000000008D
:109BA00000000000000000000000001000000000A5
:109BB0000008000800100010001000100020002015
:109BC00000000000003800440044005400440044F9
:109BD0000044003800000000001000300050001069
:109BE00000100010001000100000000000380044B9
:109BF00000440004000800100020007C0000000069
:109C00000038004400040018000400040044003838
:109C10000000000000080018002800280048007C10
:109C20000008000800000000007C004000400078B0
:109C30000004000400440038000000000038004424
:109C40000040007800440044004400380000000058
:109C5000007C0004000800100010002000200020FC
:109C60000000000000380044004400380044004474
:109C70000044003800000000003800440044004464
:109C8000003C000400440038000000000000000018
:109C900000100000000000000000001000000000A4
:109CA0000000000000000010000000000000001094
:109CB0000010001000000000000C003000400030D8
:109CC000000C000000000000000000000000007C0C
:109CD0000000007C00000000000000000000000008
:109CE0000060001800040018006000000000000080
:109CF00000380044000400080010001000000010AC
:109D00000000000000380044004C0054005C00409B
:109D10000040003800000000001000280028002843
:109D20000028007C0044004400000000007800444B
:109D30000044007800440044004400780000000023
:109D4000003800440040004000400040004400381B
:109D5000000000000070004800440044004400443B
:109D60000048007000000000007C00400040007CC3
:109D7000004000400040007C00000000007C0040EB
:109D8000004000780040004000400040000000001B
:109D90000038004400400040005C004400440038AB
:109DA00000000000004400440044007C00440044E3
:109DB00000440044000000000038001000100010B3
:109DC0000010001000100038000000000004000423
:109DD00000040004000400040044003800000000F7
:109DE0000044004800500060005000480048004413
:109DF00000000000004000400040004000400040E3
:109E00000040007C000000000044006C006C005426
:109E1000004400440044004400000000004400648A
:109E2000006400540054004C004C0044000000004A
:109E3000003800440044004400440044004400381A
:109E40000000000000780044004400440078004016
:109E5000004000400000000000380044004400447E
:109E6000004400440054003800040000007800441E
:109E7000004400440078004800480044000000000E
:109E8000003800440040003000080004004400385E
:109E900000000000007C00100010001000100010F6
:109EA0000010001000000000004400440044004482
:109EB0000044004400440038000000000044004416
:109EC00000440028002800280010001000000000B6
:109ED00000440044005400540054006C0028002842
:109EE0000000000000440028002800100010002896
:109EF000002800440000000000440044002800281E
:109F0000001000100010001000000000007C000491
:109F100000080010001000200040007C000000003D
:109F200000180010001000100010001000100010A9
:109F30000010001800200020001000100010001079
:109F400000080008000000000030001000100010A1
:109F50000010001000100010001000300010002849
:109F60000028004400000000000000000000000085
:109F700000000000000000000000000000000000E1
:109F8000000000FE002000100000000000000000A3
:109F90000000000000000000000000000038004445
:109FA000003C0044004C0034000000000040004031
:109FB00000580064004400440064005800000000A1
:109FC0000000000000380044004000400044003819
:109FD00000000000000400040034004C0044004471
:109FE000004C003400000000000000000038004475
:109FF000007C00400044003800000000000C00100D
:10A00000007C001000100010001000100000000084
:10A01000000000000034004C00440044004C0034B8
:10A0200000040078004000400058006400440044F0
:10A030000044004400000000001000000070001008
:10A0400000100010001000100000000000100000C0
:10A05000007000100010001000100010001000E050
:10A06000004000400048005000600050004800449C
:10A070000000000000700010001000100010001020
:10A0800000100010000000000000000000780054E4
:10A090000054005400540054000000000000000070
:10A0A00000580064004400440044004400000000E4
:10A0B0000000000000380044004400440044003820
:10A0C000000000000000000000580064004400444C
:10A0D0000064005800400040000000000034004CC4
:10A0E00000440044004C0034000400040000000060
:10A0F00000580064004000400040004000000000A4
:10A10000000000000038004400300008004400381F
:10A110000000000000200020007800200020002027
:10A12000002000180000000000000000004400446F
:10A1300000440044004C0034000000000000000017
:10A1400000440044002800280028001000000000FF
:10A1500000000000005400540054006C0028002847
:10A160000000000000000000004400280010001063
:10A1700000280044000000000000000000440044EB
:10A1800000280028001000100010006000000000EF
:10A19000007C0008001000200040007C000000004F
:10A1A0000018001000100010002000200010001007
:10A1B0000010001800100010001000100010001017
:10A1C00000100010001000100030001000100010EF
:10A1D000000800080010001000100030000000000F
:10A1E00000000074004C00000000000000000000AF
:10A1F000816807E002681168536889185B18C360BA
:10A2000008320260C2689142F4D04A1C8260087829
:10A2100070472DE9FF4D00F1080100914FF0000A51
:10A220000168009A490802EBC1010191D34600215F
:10A23000029103910168490800EBC101406800F0F8
:10A24000010501F10804400804EBC0061FE000A866
:10A25000FFF7CEFF47B200A8FFF7CAFF8046DA45F6
:10A260000DD1B44208BF00F01BF8D4F800A005B12E
:10A27000CA44606800EB0A0B0834DA45F1D00AF8EA
:10A28000018B002F09D57F1CE9D1DA45DFD1B4421B
:10A29000DDD1304604B0BDE8F08D7F1EDBD5F4E79C
:10A2A000012000F001B8000080B5C046C046024A57
:10A2B00011001820ABBEFBE72600020010B50749CD
:10A2C00079441831064C7C44163404E00A68081DB1
:10A2D000511888470146A142F8D110BD080000007E
:10A2E00030000000D380FFFFC003000024010020E5
:10A2F000000000001FFFFFFF02000000020000003E
:10A30000D402000031000000000000202101000004
:10A31000534F4654574152452056455253494F4E8C
:10A320005F30312F32342E30392E313500000000AD
:10A330003D3D3D3D3D3D3D3D3D3D3D3D3D3D3D3D4D
:10A340003D3D3D3D3D3D3D3D3D3D3D3D0000000031
:10A3500000F009F8002801D0FFF7B0FF0020F5F762
:10A36000E5FF00F002F80120704700F001B800009E
:10A3700007463846FFF798FFFBE70000322E2046DD
:10A38000414E205357495443482D3E204F4E000024
:10A39000332E205445524D4F4D455452202D3E20D2
:10A3A00000000000504F57455220535550504C412B
:10A3B00059000000496E697469616C697A61746959
:10A3C0006F6E3A00312E43616C6962726174696F1D
:10A3D0006E205600322E43616C6962726174696F3F
:10A3E0006E204100332E50726F74656374204343B6
:10A3F0002F435600312E2044415441464C4153488E
:10A40000202D3E000148804701480047B927000839
:10A4100051A4000830302E303030205600000000AB
:10A4200030302E3030303020410000002D2D2E2DC8
:10A430002D2D2D2041000000352E536176652F45CE
:10A440007869740030303A30303A30303A30300089
:10A45000C046C046C046C046FFF77AFF302E3030B7
:10A4600030300000302E30303030000025312E34B6
:10A470006600000078313030000000007831303064
:10A48000300000007831303030300000783130203A
:10A49000202000007831303020200000783130302A
:10A4A000302000002530336425000000204D616914
:10A4B0006E20200020416D7065722000204368618D
:10A4C00072672000204D656E752000004C6F61643E
:10A4D00000000000566F6C7461676500437572720E
:10A4E000656E74007831303030300000342E4265B3
:10A4F0006570000025312E3466000000FFF7FEBFB6
:10A50000FFF7FEBFFFF7FEBFFFF7FEBFFFF7FEBF7F
:10A51000FFF7FEBFFFF7FEBFFFF7FEBFFFF7FEBF6F
:10A52000FFF7FEBFFFF7FEBFFFF7FEBFFFF7FEBF5F
:10A53000FFF7FEBFFFF7FEBFFFF7FEBFFFF7FEBF4F
:10A54000F5F781BEFFF7FEBFFFF7FEBFF5F7D2BDFF
:10A55000FFF7FEBFFFF7FEBFFFF7FEBFFFF7FEBF2F
:10A56000FFF7FEBFFFF7FEBFFFF7FEBFFFF7FEBF1F
:10A57000FFF7FEBFFFF7FEBFFFF7FEBFFFF7FEBF0F
:10A58000FFF7FEBFFFF7FEBFFFF7FEBFFFF7FEBFFF
:10A59000FFF7FEBFFFF7FEBFF5F70ABEFFF7FEBFEE
:10A5A000FFF7FEBFFFF7FEBFFFF7FEBFFFF7FEBFDF
:10A5B000FFF7FEBFFFF7FEBFFFF7FEBFFFF7FEBFCF
:10A5C000F5F75CBEFFF7FEBFFFF7FEBFFFF7FEBF6C
:10A5D000FFF7FEBFE400F8FFDC00FAFF8100D100C6
:10A5E0001F070A0000849A00080B120000288D0043
:10A5F00008101A0000DC7900080000803F0000808D
:08A600003FFC00000100000016
:040000050800A451FA
:00000001FF
